:06000000028376028DD0A0
:03000B000287A7C2
:03001300028DF665
:1000230002849A900A58EBF0A3EAF0A3E9F07B006C
:100033007A007900900A58EBF0A3EAF0A3E9F022E2
:100043000281B4C2D5E830E70FB2D5E4C39BFBE429
:100053009AFAE499F9E498F8EC30E717B2D512006C
:100063007C12519FE4C39BFBE49AFAE499F9E49868
:10007300F8800312519F30D50DE4C39FFFE49EFE29
:07008300E49DFDE49CFC225A
:03008B00028408E4
:1000930002824B900278EBF0A3EAF0A3E9F090021E
:1000A30078E0FBA3E0FAA3E0F912528B90027E12F0
:1000B3005339900278E0FBA3E0FAA3E0F9758204D8
:1000C3007583001252AB900282125339900278E08A
:1000D300FBA3E0FAA3E0F97582087583001252AB23
:1000E300900286125339900278E0FBA3E0FAA3E072
:1000F300F975820C7583001252AB90028A12533940
:100103007B017A02798EC003C002C00190027BE0BA
:10011300FBA3E0FAA3E0F99008C5EBF0A3EAF0A390
:10012300E9F09008C812534500000040D001D00206
:10013300D003126CAE90027EE0F8A3E0F9A3E0FADC
:10014300A3E0FBC000C001C002C003900282E0FC38
:10015300A3E0FDA3E0FEA3E0FF12523190028AE088
:10016300F8A3E0F9A3E0FAA3E0FBEF5BFFEE5AFE8E
:10017300ED59FDEC58FCC004C005C006C007900251
:1001830086E0FCA3E0FDA3E0FEA3E0FF900282E093
:10019300F8A3E0F9A3E0FAA3E0FBEB5FFFEA5EFE5E
:1001A300E95DFDE85CFCD003D002D001D000EF4B49
:1001B300FFEE4AFEED49FDEC48FC90028EE0F8A309
:1001C300E0F9A3E0FAA3E0FBEF2BFFEE3AFEED39F3
:1001D300FDEC38FCEF2478FFEE34A4FEED346AFD29
:1001E300EC34D7FCD003D002D001D000EB2FFFEAD0
:1001F3003EFEE93DFDE83CFC90027E12533990023D
:100203007EE0FCA3E0FDA3E0FEA3E0FF780712522B
:1002130078C004C005C006C00790027EE0FCA3E0DE
:10022300FDA3E0FEA3E0FF7819125265A804A90517
:10023300AA06AB07D007D006D005D004EB4FFFEAE0
:100243004EFEE94DFDE84CFC90027E1253399002BC
:100253007EE0FCA3E0FDA3E0FEA3E0FF900282E0CA
:10026300F8A3E0F9A3E0FAA3E0FBEF2BFFEE3AFEDD
:10027300ED39FDEC38FC90027E12533990028AE08E
:10028300F8A3E0F9A3E0FAA3E0FBC000C001C002B9
:10029300C00390027EE0FCA3E0FDA3E0FEA3E0FF29
:1002A300125231900286E0F8A3E0F9A3E0FAA3E04A
:1002B300FBEF5BFFEE5AFEED59FDEC58FCC004C0AA
:1002C30005C006C007900282E0FCA3E0FDA3E0FEA8
:1002D300A3E0FF90027EE0F8A3E0F9A3E0FAA3E035
:1002E300FBEB5FFFEA5EFEE95DFDE85CFCD003D05B
:1002F30002D001D000EF4BFFEE4AFEED49FDEC4882
:10030300FC900292E0F8A3E0F9A3E0FAA3E0FBEF8C
:100313002BFFEE3AFEED39FDEC38FCEF2456FFEEF1
:1003230034B7FEED34C7FDEC34E8FCD003D002D083
:1003330001D000EB2FFFEA3EFEE93DFDE83CFC90D7
:10034300028A12533990028AE0FCA3E0FDA3E0FE87
:10035300A3E0FF780C125278C004C005C006C007A2
:1003630090028AE0FCA3E0FDA3E0FEA3E0FF781483
:10037300125265A804A905AA06AB07D007D006D078
:1003830005D004EB4FFFEA4EFEE94DFDE84CFC902F
:10039300028A12533990028AE0FCA3E0FDA3E0FE37
:1003A300A3E0FF90027EE0F8A3E0F9A3E0FAA3E064
:1003B300FBEF2BFFEE3AFEED39FDEC38FC90028AA1
:1003C300125339900286E0F8A3E0F9A3E0FAA3E020
:1003D300FBC000C001C002C00390028AE0FCA3E09E
:1003E300FDA3E0FEA3E0FF125231900282E0F8A3E6
:1003F300E0F9A3E0FAA3E0FBEF5BFFEE5AFEED5951
:10040300FDEC58FCC004C005C006C00790027EE0A6
:10041300FCA3E0FDA3E0FEA3E0FF90028AE0F8A3C3
:10042300E0F9A3E0FAA3E0FBEB5FFFEA5EFEE95D20
:10043300FDE85CFCD003D002D001D000EF4BFFEE0F
:100443004AFEED49FDEC48FC900296E0F8A3E0F982
:10045300A3E0FAA3E0FBEF2BFFEE3AFEED39FDEC50
:1004630038FCEF24DBFFEE3470FEED3420FDEC347A
:1004730024FCD003D002D001D000EB2FFFEA3EFED4
:10048300E93DFDE83CFC900286125339900286E078
:10049300FCA3E0FDA3E0FEA3E0FF7811125278C0B5
:1004A30004C005C006C007900286E0FCA3E0FDA3DC
:1004B300E0FEA3E0FF780F125265A804A905AA067F
:1004C300AB07D007D006D005D004EB4FFFEA4EFEB2
:1004D300E94DFDE84CFC900286125339900286E008
:1004E300FCA3E0FDA3E0FEA3E0FF90028AE0F8A3F3
:1004F300E0F9A3E0FAA3E0FBEF2BFFEE3AFEED39C0
:10050300FDEC38FC900286125339900282E0F8A386
:10051300E0F9A3E0FAA3E0FBC000C001C002C003FE
:10052300900286E0FCA3E0FDA3E0FEA3E0FF1252ED
:100533003190027EE0F8A3E0F9A3E0FAA3E0FBEF39
:100543005BFFEE5AFEED59FDEC58FCC004C005C03C
:1005530006C00790028AE0FCA3E0FDA3E0FEA3E04F
:10056300FF900286E0F8A3E0F9A3E0FAA3E0FBEB37
:100573005FFFEA5EFEE95DFDE85CFCD003D002D0DC
:1005830001D000EF4BFFEE4AFEED49FDEC48FC9035
:10059300029AE0F8A3E0F9A3E0FAA3E0FBEF2BFF54
:1005A300EE3AFEED39FDEC38FCEF24EEFFEE34CEEF
:1005B300FEED34BDFDEC34C1FCD003D002D001D03C
:1005C30000EB2FFFEA3EFEE93DFDE83CFC90028292
:1005D300125339900282E0FCA3E0FDA3E0FEA3E006
:1005E300FF7816125278C004C005C006C0079002F7
:1005F30082E0FCA3E0FDA3E0FEA3E0FF780A125231
:1006030065A804A905AA06AB07D007D006D005D074
:1006130004EB4FFFEA4EFEE94DFDE84CFC900282ED
:10062300125339900282E0FCA3E0FDA3E0FEA3E0B5
:10063300FF900286E0F8A3E0F9A3E0FAA3E0FBEF62
:100643002BFFEE3AFEED39FDEC38FC90028212539B
:100653003990027EE0F8A3E0F9A3E0FAA3E0FBC03F
:1006630000C001C002C003900282E0FCA3E0FDA32E
:10067300E0FEA3E0FF12523190028AE0F8A3E0F912
:10068300A3E0FAA3E0FBEF5BFFEE5AFEED59FDECAE
:1006930058FCC004C005C006C007900286E0FCA356
:1006A300E0FDA3E0FEA3E0FF900282E0F8A3E0F9FF
:1006B300A3E0FAA3E0FBEB5FFFEA5EFEE95DFDE882
:1006C3005CFCD003D002D001D000EF4BFFEE4AFE1A
:1006D300ED49FDEC48FC90029EE0F8A3E0F9A3E0AD
:1006E300FAA3E0FBEF2BFFEE3AFEED39FDEC38FC0D
:1006F300EF24AFFFEE340FFEED347CFDEC34F5FC5C
:10070300D003D002D001D000EB2FFFEA3EFEE93D3B
:10071300FDE83CFC90027E12533990027EE0FCA37C
:10072300E0FDA3E0FEA3E0FF7807125278C004C007
:1007330005C006C00790027EE0FCA3E0FDA3E0FE37
:10074300A3E0FF7819125265A804A905AA06AB070E
:10075300D007D006D005D004EB4FFFEA4EFEE94D9B
:10076300FDE84CFC90027E12533990027EE0FCA31C
:10077300E0FDA3E0FEA3E0FF900282E0F8A3E0F92E
:10078300A3E0FAA3E0FBEF2BFFEE3AFEED39FDEC1D
:1007930038FC90027E12533990028AE0F8A3E0F904
:1007A300A3E0FAA3E0FBC000C001C002C0039002B3
:1007B3007EE0FCA3E0FDA3E0FEA3E0FF1252319034
:1007C3000286E0F8A3E0F9A3E0FAA3E0FBEF5BFF06
:1007D300EE5AFEED59FDEC58FCC004C005C006C03E
:1007E30007900282E0FCA3E0FDA3E0FEA3E0FF90FC
:1007F300027EE0F8A3E0F9A3E0FAA3E0FBEB5FFFDE
:10080300EA5EFEE95DFDE85CFCD003D002D001D0D6
:1008130000EF4BFFEE4AFEED49FDEC48FC9002A2CF
:10082300E0F8A3E0F9A3E0FAA3E0FBEF2BFFEE3A35
:10083300FEED39FDEC38FCEF242AFFEE34C6FEED65
:100843003487FDEC3447FCD003D002D001D000EB59
:100853002FFFEA3EFEE93DFDE83CFC90028A12537D
:100863003990028AE0FCA3E0FDA3E0FEA3E0FF7859
:100873000C125278C004C005C006C00790028AE07B
:10088300FCA3E0FDA3E0FEA3E0FF7814125265A8E9
:1008930004A905AA06AB07D007D006D005D004EB00
:1008A3004FFFEA4EFEE94DFDE84CFC90028A1253DD
:1008B3003990028AE0FCA3E0FDA3E0FEA3E0FF90F1
:1008C300027EE0F8A3E0F9A3E0FAA3E0FBEF2BFF3D
:1008D300EE3AFEED39FDEC38FC90028A1253399062
:1008E3000286E0F8A3E0F9A3E0FAA3E0FBC000C0AE
:1008F30001C002C00390028AE0FCA3E0FDA3E0FE76
:10090300A3E0FF125231900282E0F8A3E0F9A3E0E2
:10091300FAA3E0FBEF5BFFEE5AFEED59FDEC58FC4A
:10092300C004C005C006C00790027EE0FCA3E0FD42
:10093300A3E0FEA3E0FF90028AE0F8A3E0F9A3E0BE
:10094300FAA3E0FBEB5FFFEA5EFEE95DFDE85CFC1A
:10095300D003D002D001D000EF4BFFEE4AFEED49A9
:10096300FDEC48FC9002A6E0F8A3E0F9A3E0FAA3AB
:10097300E0FBEF2BFFEE3AFEED39FDEC38FCEF2404
:1009830013FFEE3446FEED3430FDEC34A8FCD00307
:10099300D002D001D000EB2FFFEA3EFEE93DFDE897
:1009A3003CFC900286125339900286E0FCA3E0FDE2
:1009B300A3E0FEA3E0FF7811125278C004C005C083
:1009C30006C007900286E0FCA3E0FDA3E0FEA3E0DF
:1009D300FF780F125265A804A905AA06AB07D00732
:1009E300D006D005D004EB4FFFEA4EFEE94DFDE8FB
:1009F3004CFC900286125339900286E0FCA3E0FD82
:100A0300A3E0FEA3E0FF90028AE0F8A3E0F9A3E0ED
:100A1300FAA3E0FBEF2BFFEE3AFEED39FDEC38FCD9
:100A2300900286125339900282E0F8A3E0F9A3E022
:100A3300FAA3E0FBC000C001C002C003900286E03D
:100A4300FCA3E0FDA3E0FEA3E0FF12523190027E7F
:100A5300E0F8A3E0F9A3E0FAA3E0FBEF5BFFEE5AB3
:100A6300FEED59FDEC58FCC004C005C006C007905C
:100A7300028AE0FCA3E0FDA3E0FEA3E0FF90028670
:100A8300E0F8A3E0F9A3E0FAA3E0FBEB5FFFEA5E83
:100A9300FEE95DFDE85CFCD003D002D001D000EF9D
:100AA3004BFFEE4AFEED49FDEC48FC9002AAE0F84C
:100AB300A3E0F9A3E0FAA3E0FBEF2BFFEE3AFEED90
:100AC30039FDEC38FCEF2401FFEE3495FEED34469E
:100AD300FDEC34FDFCD003D002D001D000EB2FFF9E
:100AE300EA3EFEE93DFDE83CFC9002821253399058
:100AF3000282E0FCA3E0FDA3E0FEA3E0FF78161270
:100B03005278C004C005C006C007900282E0FCA36F
:100B1300E0FDA3E0FEA3E0FF780A125265A804A952
:100B230005AA06AB07D007D006D005D004EB4FFFCC
:100B3300EA4EFEE94DFDE84CFC90028212533990D7
:100B43000282E0FCA3E0FDA3E0FEA3E0FF900286A7
:100B5300E0F8A3E0F9A3E0FAA3E0FBEF2BFFEE3A02
:100B6300FEED39FDEC38FC90028212533990027E7F
:100B7300E0F8A3E0F9A3E0FAA3E0FBC000C001C0E2
:100B830002C003900282E0FCA3E0FDA3E0FEA3E029
:100B9300FF12523190028AE0F8A3E0F9A3E0FAA32E
:100BA300E0FBEF5BFFEE5AFEED59FDEC58FCC00491
:100BB300C005C006C007900286E0FCA3E0FDA3E0E9
:100BC300FEA3E0FF900282E0F8A3E0F9A3E0FAA31A
:100BD300E0FBEB5FFFEA5EFEE95DFDE85CFCD00352
:100BE300D002D001D000EF4BFFEE4AFEED49FDEC01
:100BF30048FC9002AEE0F8A3E0F9A3E0FAA3E0FB1F
:100C0300EF2BFFEE3AFEED39FDEC38FCEF24D8FF75
:100C1300EE3498FEED3480FDEC3469FCD003D00251
:100C2300D001D000EB2FFFEA3EFEE93DFDE83CFC9E
:100C330090027E12533990027EE0FCA3E0FDA3E014
:100C4300FEA3E0FF7807125278C004C005C006C0B7
:100C53000790027EE0FCA3E0FDA3E0FEA3E0FF78A3
:100C630019125265A804A905AA06AB07D007D00636
:100C7300D005D004EB4FFFEA4EFEE94DFDE84CFCF6
:100C830090027E12533990027EE0FCA3E0FDA3E0C4
:100C9300FEA3E0FF900282E0F8A3E0F9A3E0FAA349
:100CA300E0FBEF2BFFEE3AFEED39FDEC38FC900252
:100CB3007E12533990028AE0F8A3E0F9A3E0FAA385
:100CC300E0FBC000C001C002C00390027EE0FCA3B1
:100CD300E0FDA3E0FEA3E0FF125231900286E0F8AC
:100CE300A3E0F9A3E0FAA3E0FBEF5BFFEE5AFEED0E
:100CF30059FDEC58FCC004C005C006C00790028231
:100D0300E0FCA3E0FDA3E0FEA3E0FF90027EE0F899
:100D1300A3E0F9A3E0FAA3E0FBEB5FFFEA5EFEE9E1
:100D23005DFDE85CFCD003D002D001D000EF4BFFA7
:100D3300EE4AFEED49FDEC48FC9002B2E0F8A3E078
:100D4300F9A3E0FAA3E0FBEF2BFFEE3AFEED39FD4A
:100D5300EC38FCEF24AFFFEE34F7FEED3444FDEC4A
:100D6300348BFCD003D002D001D000EB2FFFEA3E3E
:100D7300FEE93DFDE83CFC90028A12533990028A59
:100D8300E0FCA3E0FDA3E0FEA3E0FF780C125278A1
:100D9300C004C005C006C00790028AE0FCA3E0FDC2
:100DA300A3E0FEA3E0FF7814125265A804A905AAE4
:100DB30006AB07D007D006D005D004EB4FFFEA4EB1
:100DC300FEE94DFDE84CFC90028A12533990028AE9
:100DD300E0FCA3E0FDA3E0FEA3E0FF90027EE0F8C9
:100DE300A3E0F9A3E0FAA3E0FBEF2BFFEE3AFEED5D
:100DF30039FDEC38FC90028A125339900286E0F8F0
:100E0300A3E0F9A3E0FAA3E0FBC000C001C002C065
:100E13000390028AE0FCA3E0FDA3E0FEA3E0FF123F
:100E23005231900282E0F8A3E0F9A3E0FAA3E0FBD9
:100E3300EF5BFFEE5AFEED59FDEC58FCC004C00514
:100E4300C006C00790027EE0FCA3E0FDA3E0FEA382
:100E5300E0FF90028AE0F8A3E0F9A3E0FAA3E0FB45
:100E6300EB5FFFEA5EFEE95DFDE85CFCD003D002C8
:100E7300D001D000EF4BFFEE4AFEED49FDEC48FCFC
:100E83009002B6E0F8A3E0F9A3E0FAA3E0FBEF2BAE
:100E9300FFEE3AFEED39FDEC38FCEF24B1FFEE3402
:100EA3005BFEED34FFFDEC34FFFCD003D002D00138
:100EB300D000EB2FFFEA3EFEE93DFDE83CFC90024B
:100EC30086125339900286E0FCA3E0FDA3E0FEA363
:100ED300E0FF7811125278C004C005C006C0079025
:100EE3000286E0FCA3E0FDA3E0FEA3E0FF780F127F
:100EF3005265A804A905AA06AB07D007D006D005FA
:100F0300D004EB4FFFEA4EFEE94DFDE84CFC9002A6
:100F130086125339900286E0FCA3E0FDA3E0FEA312
:100F2300E0FF90028AE0F8A3E0F9A3E0FAA3E0FB74
:100F3300EF2BFFEE3AFEED39FDEC38FC9002861202
:100F43005339900282E0F8A3E0F9A3E0FAA3E0FBAF
:100F5300C000C001C002C003900286E0FCA3E0FD14
:100F6300A3E0FEA3E0FF12523190027EE0F8A3E07B
:100F7300F9A3E0FAA3E0FBEF5BFFEE5AFEED59FDA8
:100F8300EC58FCC004C005C006C00790028AE0FC10
:100F9300A3E0FDA3E0FEA3E0FF900286E0F8A3E058
:100FA300F9A3E0FAA3E0FBEB5FFFEA5EFEE95DFD78
:100FB300E85CFCD003D002D001D000EF4BFFEE4A37
:100FC300FEED49FDEC48FC9002BAE0F8A3E0F9A37A
:100FD300E0FAA3E0FBEF2BFFEE3AFEED39FDEC3830
:100FE300FCEF24BEFFEE34D7FEED345CFDEC348918
:100FF300FCD003D002D001D000EB2FFFEA3EFEE984
:101003003DFDE83CFC900282125339900282E0FCE1
:10101300A3E0FDA3E0FEA3E0FF7816125278C0041C
:10102300C005C006C007900282E0FCA3E0FDA3E078
:10103300FEA3E0FF780A125265A804A905AA06AB2D
:1010430007D007D006D005D004EB4FFFEA4EFEE9E8
:101053004DFDE84CFC900282125339900282E0FC71
:10106300A3E0FDA3E0FEA3E0FF900286E0F8A3E087
:10107300F9A3E0FAA3E0FBEF2BFFEE3AFEED39FD17
:10108300EC38FC90028212533990027EE0F8A3E020
:10109300F9A3E0FAA3E0FBC000C001C002C00390C3
:1010A3000282E0FCA3E0FDA3E0FEA3E0FF125231C5
:1010B30090028AE0F8A3E0F9A3E0FAA3E0FBEF5B78
:1010C300FFEE5AFEED59FDEC58FCC004C005C00606
:1010D300C007900286E0FCA3E0FDA3E0FEA3E0FFCF
:1010E300900282E0F8A3E0F9A3E0FAA3E0FBEB5F50
:1010F300FFEA5EFEE95DFDE85CFCD003D002D001AF
:10110300D000EF4BFFEE4AFEED49FDEC48FC9002A8
:10111300BEE0F8A3E0F9A3E0FAA3E0FBEF2BFFEEB8
:101123003AFEED39FDEC38FCEF2422FFEE3411FEDC
:10113300ED3490FDEC346BFCD003D002D001D00031
:10114300EB2FFFEA3EFEE93DFDE83CFC90027E12F8
:10115300533990027EE0FCA3E0FDA3E0FEA3E0FF91
:101163007807125278C004C005C006C00790027EFB
:10117300E0FCA3E0FDA3E0FEA3E0FF7819125265B3
:10118300A804A905AA06AB07D007D006D005D0044A
:10119300EB4FFFEA4EFEE94DFDE84CFC90027E1258
:1011A300533990027EE0FCA3E0FDA3E0FEA3E0FF41
:1011B300900282E0F8A3E0F9A3E0FAA3E0FBEF2BAF
:1011C300FFEE3AFEED39FDEC38FC90027E12533906
:1011D30090028AE0F8A3E0F9A3E0FAA3E0FBC000E1
:1011E300C001C002C00390027EE0FCA3E0FDA3E0C7
:1011F300FEA3E0FF125231900286E0F8A3E0F9A3C8
:10120300E0FAA3E0FBEF5BFFEE5AFEED59FDEC586D
:10121300FCC004C005C006C007900282E0FCA3E046
:10122300FDA3E0FEA3E0FF90027EE0F8A3E0F9A3B4
:10123300E0FAA3E0FBEB5FFFEA5EFEE95DFDE85C3D
:10124300FCD003D002D001D000EF4BFFEE4AFEEDFD
:1012530049FDEC48FC9002C2E0F8A3E0F9A3E0FAF0
:10126300A3E0FBEF2BFFEE3AFEED39FDEC38FCEF8C
:101273002493FFEE3471FEED3498FDEC34FDFCD085
:1012830003D002D001D000EB2FFFEA3EFEE93DFD83
:10129300E83CFC90028A12533990028AE0FCA3E0F6
:1012A300FDA3E0FEA3E0FF780C125278C004C00552
:1012B300C006C00790028AE0FCA3E0FDA3E0FEA302
:1012C300E0FF7814125265A804A905AA06AB07D05B
:1012D30007D006D005D004EB4FFFEA4EFEE94DFDE3
:1012E300E84CFC90028A12533990028AE0FCA3E096
:1012F300FDA3E0FEA3E0FF90027EE0F8A3E0F9A3E4
:10130300E0FAA3E0FBEF2BFFEE3AFEED39FDEC38FC
:10131300FC90028A125339900286E0F8A3E0F9A305
:10132300E0FAA3E0FBC000C001C002C00390028A40
:10133300E0FCA3E0FDA3E0FEA3E0FF125231900224
:1013430082E0F8A3E0F9A3E0FAA3E0FBEF5BFFEE92
:101353005AFEED59FDEC58FCC004C005C006C00799
:1013630090027EE0FCA3E0FDA3E0FEA3E0FF900279
:101373008AE0F8A3E0F9A3E0FAA3E0FBEB5FFFEA5E
:101383005EFEE95DFDE85CFCD003D002D001D00035
:10139300EF4BFFEE4AFEED49FDEC48FC9002C6E040
:1013A300F8A3E0F9A3E0FAA3E0FBEF2BFFEE3AFE8C
:1013B300ED39FDEC38FCEF248EFFEE3443FEED34C3
:1013C30079FDEC34A6FCD003D002D001D000EB2F82
:1013D300FFEA3EFEE93DFDE83CFC900286125339EC
:1013E300900286E0FCA3E0FDA3E0FEA3E0FF7811FA
:1013F300125278C004C005C006C007900286E0FC04
:10140300A3E0FDA3E0FEA3E0FF780F125265A8045A
:10141300A905AA06AB07D007D006D005D004EB4F29
:10142300FFEA4EFEE94DFDE84CFC9002861253396B
:10143300900286E0FCA3E0FDA3E0FEA3E0FF9002A0
:101443008AE0F8A3E0F9A3E0FAA3E0FBEF2BFFEEB9
:101453003AFEED39FDEC38FC9002861253399002C6
:1014630082E0F8A3E0F9A3E0FAA3E0FBC000C00127
:10147300C002C003900286E0FCA3E0FDA3E0FEA34C
:10148300E0FF12523190027EE0F8A3E0F9A3E0FA04
:10149300A3E0FBEF5BFFEE5AFEED59FDEC58FCC0F9
:1014A30004C005C006C00790028AE0FCA3E0FDA3C8
:1014B300E0FEA3E0FF900286E0F8A3E0F9A3E0FAE0
:1014C300A3E0FBEB5FFFEA5EFEE95DFDE85CFCD0B9
:1014D30003D002D001D000EF4BFFEE4AFEED49FDF1
:1014E300EC48FC9002CAE0F8A3E0F9A3E0FAA3E019
:1014F300FBEF2BFFEE3AFEED39FDEC38FCEF242138
:10150300FFEE3408FEED34B4FDEC3449FCD003D0D7
:1015130002D001D000EB2FFFEA3EFEE93DFDE83C9F
:10152300FC900282125339900282E0FCA3E0FDA3F7
:10153300E0FEA3E0FF7816125278C004C005C0068F
:10154300C007900282E0FCA3E0FDA3E0FEA3E0FF5E
:10155300780A125265A804A905AA06AB07D007D0DA
:1015630006D005D004EB4FFFEA4EFEE94DFDE84CF3
:10157300FC900282125339900282E0FCA3E0FDA3A7
:10158300E0FEA3E0FF900286E0F8A3E0F9A3E0FA0F
:10159300A3E0FBEF2BFFEE3AFEED39FDEC38FC90B8
:1015A300028212533990027EE0F8A3E0F9A3E0FA35
:1015B300A3E0FBC000C001C002C00390028AE0FCAC
:1015C300A3E0FDA3E0FEA3E0FF125231900286E008
:1015D300F8A3E0F9A3E0FAA3E0FBEF5BFFEE5AFE0A
:1015E300ED59FDEC58FCC004C005C006C0079002CD
:1015F3008AE0FCA3E0FDA3E0FEA3E0FF900282E00B
:10160300F8A3E0F9A3E0FAA3E0FBEB5FFFEA5EFED9
:10161300E95DFDE85CFCD003D002D001D000EF4BC4
:10162300FFEE4AFEED49FDEC48FC900292E0F8A380
:10163300E0F9A3E0FAA3E0FBEF2BFFEE3AFEED396E
:10164300FDEC38FCEF2462FFEE3425FEED341EFD85
:10165300EC34F6FCD003D002D001D000EB2FFFEA2C
:101663003EFEE93DFDE83CFC90027E1253399002B8
:101673007EE0FCA3E0FDA3E0FEA3E0FF78051252A9
:1016830078C004C005C006C00790027EE0FCA3E05A
:10169300FDA3E0FEA3E0FF781B125265A804A90591
:1016A300AA06AB07D007D006D005D004EB4FFFEA5C
:1016B3004EFEE94DFDE84CFC90027E125339900238
:1016C3007EE0FCA3E0FDA3E0FEA3E0FF900282E046
:1016D300F8A3E0F9A3E0FAA3E0FBEF2BFFEE3AFE59
:1016E300ED39FDEC38FC90027E12533990028AE00A
:1016F300F8A3E0F9A3E0FAA3E0FBC000C001C00235
:10170300C003900286E0FCA3E0FDA3E0FEA3E0FF9C
:10171300125231900282E0F8A3E0F9A3E0FAA3E0C9
:10172300FBEF5BFFEE5AFEED59FDEC58FCC004C025
:1017330005C006C007900286E0FCA3E0FDA3E0FE1F
:10174300A3E0FF90027EE0F8A3E0F9A3E0FAA3E0B0
:10175300FBEB5FFFEA5EFEE95DFDE85CFCD003D0D6
:1017630002D001D000EF4BFFEE4AFEED49FDEC48FD
:10177300FC9002A6E0F8A3E0F9A3E0FAA3E0FBEFF4
:101783002BFFEE3AFEED39FDEC38FCEF2440FFEE83
:1017930034B3FEED3440FDEC34C0FCD003D002D0B2
:1017A30001D000EB2FFFEA3EFEE93DFDE83CFC9053
:1017B300028A12533990028AE0FCA3E0FDA3E0FE03
:1017C300A3E0FF7809125278C004C005C006C00721
:1017D30090028AE0FCA3E0FDA3E0FEA3E0FF7817FC
:1017E300125265A804A905AA06AB07D007D006D0F4
:1017F30005D004EB4FFFEA4EFEE94DFDE84CFC90AB
:10180300028A12533990028AE0FCA3E0FDA3E0FEB2
:10181300A3E0FF90027EE0F8A3E0F9A3E0FAA3E0DF
:10182300FBEF2BFFEE3AFEED39FDEC38FC90028A1C
:10183300125339900286E0F8A3E0F9A3E0FAA3E09B
:10184300FBC000C001C002C003900282E0FCA3E021
:10185300FDA3E0FEA3E0FF12523190027EE0F8A365
:10186300E0F9A3E0FAA3E0FBEF5BFFEE5AFEED59CC
:10187300FDEC58FCC004C005C006C007900282E01E
:10188300FCA3E0FDA3E0FEA3E0FF90028AE0F8A33F
:10189300E0F9A3E0FAA3E0FBEB5FFFEA5EFEE95D9C
:1018A300FDE85CFCD003D002D001D000EF4BFFEE8B
:1018B3004AFEED49FDEC48FC9002BAE0F8A3E0F9DA
:1018C300A3E0FAA3E0FBEF2BFFEE3AFEED39FDECCC
:1018D30038FCEF2451FFEE345AFEED345EFDEC3458
:1018E30026FCD003D002D001D000EB2FFFEA3EFE4E
:1018F300E93DFDE83CFC900286125339900286E0F4
:10190300FCA3E0FDA3E0FEA3E0FF780E125278C033
:1019130004C005C006C007900286E0FCA3E0FDA357
:10192300E0FEA3E0FF7812125265A804A905AA06F7
:10193300AB07D007D006D005D004EB4FFFEA4EFE2D
:10194300E94DFDE84CFC900286125339900286E083
:10195300FCA3E0FDA3E0FEA3E0FF90028AE0F8A36E
:10196300E0F9A3E0FAA3E0FBEF2BFFEE3AFEED393B
:10197300FDEC38FC900286125339900282E0F8A302
:10198300E0F9A3E0FAA3E0FBC000C001C002C0037A
:1019930090027EE0FCA3E0FDA3E0FEA3E0FF125271
:1019A3003190028AE0F8A3E0F9A3E0FAA3E0FBEFA9
:1019B3005BFFEE5AFEED59FDEC58FCC004C005C0B8
:1019C30006C00790027EE0FCA3E0FDA3E0FEA3E0D7
:1019D300FF900286E0F8A3E0F9A3E0FAA3E0FBEBB3
:1019E3005FFFEA5EFEE95DFDE85CFCD003D002D058
:1019F30001D000EF4BFFEE4AFEED49FDEC48FC90B1
:101A0300028EE0F8A3E0F9A3E0FAA3E0FBEF2BFFDB
:101A1300EE3AFEED39FDEC38FCEF24AAFFEE34C7B5
:101A2300FEED34B6FDEC34E9FCD003D002D001D096
:101A330000EB2FFFEA3EFEE93DFDE83CFC9002820D
:101A4300125339900282E0FCA3E0FDA3E0FEA3E081
:101A5300FF7814125278C004C005C006C007900274
:101A630082E0FCA3E0FDA3E0FEA3E0FF780C1252AA
:101A730065A804A905AA06AB07D007D006D005D0F0
:101A830004EB4FFFEA4EFEE94DFDE84CFC90028269
:101A9300125339900282E0FCA3E0FDA3E0FEA3E031
:101AA300FF900286E0F8A3E0F9A3E0FAA3E0FBEFDE
:101AB3002BFFEE3AFEED39FDEC38FC900282125317
:101AC3003990027EE0F8A3E0F9A3E0FAA3E0FBC0BB
:101AD30000C001C002C00390028AE0FCA3E0FDA3A2
:101AE300E0FEA3E0FF125231900286E0F8A3E0F992
:101AF300A3E0FAA3E0FBEF5BFFEE5AFEED59FDEC2A
:101B030058FCC004C005C006C00790028AE0FCA3CD
:101B1300E0FDA3E0FEA3E0FF900282E0F8A3E0F97A
:101B2300A3E0FAA3E0FBEB5FFFEA5EFEE95DFDE8FD
:101B33005CFCD003D002D001D000EF4BFFEE4AFE95
:101B4300ED49FDEC48FC9002A2E0F8A3E0F9A3E024
:101B5300FAA3E0FBEF2BFFEE3AFEED39FDEC38FC88
:101B6300EF245DFFEE3410FEED342FFDEC34D6FC94
:101B7300D003D002D001D000EB2FFFEA3EFEE93DB7
:101B8300FDE83CFC90027E12533990027EE0FCA3F8
:101B9300E0FDA3E0FEA3E0FF7805125278C004C085
:101BA30005C006C00790027EE0FCA3E0FDA3E0FEB3
:101BB300A3E0FF781B125265A804A905AA06AB0788
:101BC300D007D006D005D004EB4FFFEA4EFEE94D17
:101BD300FDE84CFC90027E12533990027EE0FCA398
:101BE300E0FDA3E0FEA3E0FF900282E0F8A3E0F9AA
:101BF300A3E0FAA3E0FBEF2BFFEE3AFEED39FDEC99
:101C030038FC90027E12533990028AE0F8A3E0F97F
:101C1300A3E0FAA3E0FBC000C001C002C00390022E
:101C230086E0FCA3E0FDA3E0FEA3E0FF12523190A7
:101C33000282E0F8A3E0F9A3E0FAA3E0FBEF5BFF85
:101C4300EE5AFEED59FDEC58FCC004C005C006C0B9
:101C530007900286E0FCA3E0FDA3E0FEA3E0FF9073
:101C6300027EE0F8A3E0F9A3E0FAA3E0FBEB5FFF59
:101C7300EA5EFEE95DFDE85CFCD003D002D001D052
:101C830000EF4BFFEE4AFEED49FDEC48FC9002B637
:101C9300E0F8A3E0F9A3E0FAA3E0FBEF2BFFEE3AB1
:101CA300FEED39FDEC38FCEF2453FFEE3414FEED6A
:101CB3003444FDEC3402FCD003D002D001D000EB5D
:101CC3002FFFEA3EFEE93DFDE83CFC90028A1253F9
:101CD3003990028AE0FCA3E0FDA3E0FEA3E0FF78D5
:101CE30009125278C004C005C006C00790028AE0FA
:101CF300FCA3E0FDA3E0FEA3E0FF7817125265A862
:101D030004A905AA06AB07D007D006D005D004EB7B
:101D13004FFFEA4EFEE94DFDE84CFC90028A125358
:101D23003990028AE0FCA3E0FDA3E0FEA3E0FF906C
:101D3300027EE0F8A3E0F9A3E0FAA3E0FBEF2BFFB8
:101D4300EE3AFEED39FDEC38FC90028A12533990DD
:101D53000286E0F8A3E0F9A3E0FAA3E0FBC000C029
:101D630001C002C003900282E0FCA3E0FDA3E0FEF9
:101D7300A3E0FF12523190027EE0F8A3E0F9A3E062
:101D8300FAA3E0FBEF5BFFEE5AFEED59FDEC58FCC6
:101D9300C004C005C006C007900282E0FCA3E0FDBA
:101DA300A3E0FEA3E0FF90028AE0F8A3E0F9A3E03A
:101DB300FAA3E0FBEB5FFFEA5EFEE95DFDE85CFC96
:101DC300D003D002D001D000EF4BFFEE4AFEED4925
:101DD300FDEC48FC9002CAE0F8A3E0F9A3E0FAA303
:101DE300E0FBEF2BFFEE3AFEED39FDEC38FCEF2480
:101DF30081FFEE34E6FEED34A1FDEC34D8FCD003D4
:101E0300D002D001D000EB2FFFEA3EFEE93DFDE812
:101E13003CFC900286125339900286E0FCA3E0FD5D
:101E2300A3E0FEA3E0FF780E125278C004C005C001
:101E330006C007900286E0FCA3E0FDA3E0FEA3E05A
:101E4300FF7812125265A804A905AA06AB07D007AA
:101E5300D006D005D004EB4FFFEA4EFEE94DFDE876
:101E63004CFC900286125339900286E0FCA3E0FDFD
:101E7300A3E0FEA3E0FF90028AE0F8A3E0F9A3E069
:101E8300FAA3E0FBEF2BFFEE3AFEED39FDEC38FC55
:101E9300900286125339900282E0F8A3E0F9A3E09E
:101EA300FAA3E0FBC000C001C002C00390027EE0C1
:101EB300FCA3E0FDA3E0FEA3E0FF12523190028AEF
:101EC300E0F8A3E0F9A3E0FAA3E0FBEF5BFFEE5A2F
:101ED300FEED59FDEC58FCC004C005C006C00790D8
:101EE300027EE0FCA3E0FDA3E0FEA3E0FF900286F8
:101EF300E0F8A3E0F9A3E0FAA3E0FBEB5FFFEA5EFF
:101F0300FEE95DFDE85CFCD003D002D001D000EF18
:101F13004BFFEE4AFEED49FDEC48FC90029EE0F8D3
:101F2300A3E0F9A3E0FAA3E0FBEF2BFFEE3AFEED0B
:101F330039FDEC38FCEF24C8FFEE34FBFEED34D35F
:101F4300FDEC34E7FCD003D002D001D000EB2FFF2F
:101F5300EA3EFEE93DFDE83CFC90028212533990D3
:101F63000282E0FCA3E0FDA3E0FEA3E0FF781412ED
:101F73005278C004C005C006C007900282E0FCA3EB
:101F8300E0FDA3E0FEA3E0FF780C125265A804A9CC
:101F930005AA06AB07D007D006D005D004EB4FFF48
:101FA300EA4EFEE94DFDE84CFC9002821253399053
:101FB3000282E0FCA3E0FDA3E0FEA3E0FF90028623
:101FC300E0F8A3E0F9A3E0FAA3E0FBEF2BFFEE3A7E
:101FD300FEED39FDEC38FC90028212533990027EFB
:101FE300E0F8A3E0F9A3E0FAA3E0FBC000C001C05E
:101FF30002C00390028AE0FCA3E0FDA3E0FEA3E09D
:10200300FF125231900286E0F8A3E0F9A3E0FAA3AD
:10201300E0FBEF5BFFEE5AFEED59FDEC58FCC0040C
:10202300C005C006C00790028AE0FCA3E0FDA3E060
:10203300FEA3E0FF900282E0F8A3E0F9A3E0FAA395
:10204300E0FBEB5FFFEA5EFEE95DFDE85CFCD003CD
:10205300D002D001D000EF4BFFEE4AFEED49FDEC7C
:1020630048FC9002B2E0F8A3E0F9A3E0FAA3E0FB96
:10207300EF2BFFEE3AFEED39FDEC38FCEF24E6FFE3
:10208300EE34CDFEED34E1FDEC3421FCD003D0027F
:10209300D001D000EB2FFFEA3EFEE93DFDE83CFC1A
:1020A30090027E12533990027EE0FCA3E0FDA3E090
:1020B300FEA3E0FF7805125278C004C005C006C035
:1020C3000790027EE0FCA3E0FDA3E0FEA3E0FF781F
:1020D3001B125265A804A905AA06AB07D007D006B0
:1020E300D005D004EB4FFFEA4EFEE94DFDE84CFC72
:1020F30090027E12533990027EE0FCA3E0FDA3E040
:10210300FEA3E0FF900282E0F8A3E0F9A3E0FAA3C4
:10211300E0FBEF2BFFEE3AFEED39FDEC38FC9002CD
:102123007E12533990028AE0F8A3E0F9A3E0FAA300
:10213300E0FBC000C001C002C003900286E0FCA324
:10214300E0FDA3E0FEA3E0FF125231900282E0F82B
:10215300A3E0F9A3E0FAA3E0FBEF5BFFEE5AFEED89
:1021630059FDEC58FCC004C005C006C007900286A8
:10217300E0FCA3E0FDA3E0FEA3E0FF90027EE0F815
:10218300A3E0F9A3E0FAA3E0FBEB5FFFEA5EFEE95D
:102193005DFDE85CFCD003D002D001D000EF4BFF23
:1021A300EE4AFEED49FDEC48FC9002C6E0F8A3E0E0
:1021B300F9A3E0FAA3E0FBEF2BFFEE3AFEED39FDC6
:1021C300EC38FCEF24D6FFEE3407FEED3437FDEC9C
:1021D30034C3FCD003D002D001D000EB2FFFEA3E82
:1021E300FEE93DFDE83CFC90028A12533990028AD5
:1021F300E0FCA3E0FDA3E0FEA3E0FF780912527820
:10220300C004C005C006C00790028AE0FCA3E0FD3D
:10221300A3E0FEA3E0FF7817125265A804A905AA5C
:1022230006AB07D007D006D005D004EB4FFFEA4E2C
:10223300FEE94DFDE84CFC90028A12533990028A64
:10224300E0FCA3E0FDA3E0FEA3E0FF90027EE0F844
:10225300A3E0F9A3E0FAA3E0FBEF2BFFEE3AFEEDD8
:1022630039FDEC38FC90028A125339900286E0F86B
:10227300A3E0F9A3E0FAA3E0FBC000C001C002C0E1
:1022830003900282E0FCA3E0FDA3E0FEA3E0FF12C3
:10229300523190027EE0F8A3E0F9A3E0FAA3E0FB59
:1022A300EF5BFFEE5AFEED59FDEC58FCC004C00590
:1022B300C006C007900282E0FCA3E0FDA3E0FEA3FA
:1022C300E0FF90028AE0F8A3E0F9A3E0FAA3E0FBC1
:1022D300EB5FFFEA5EFEE95DFDE85CFCD003D00244
:1022E300D001D000EF4BFFEE4AFEED49FDEC48FC78
:1022F30090029AE0F8A3E0F9A3E0FAA3E0FBEF2B46
:10230300FFEE3AFEED39FDEC38FCEF2487FFEE34A7
:102313000DFEED34D5FDEC34F4FCD003D002D00136
:10232300D000EB2FFFEA3EFEE93DFDE83CFC9002C6
:1023330086125339900286E0FCA3E0FDA3E0FEA3DE
:10234300E0FF780E125278C004C005C006C00790A3
:102353000286E0FCA3E0FDA3E0FEA3E0FF781212F7
:102363005265A804A905AA06AB07D007D006D00575
:10237300D004EB4FFFEA4EFEE94DFDE84CFC900222
:1023830086125339900286E0FCA3E0FDA3E0FEA38E
:10239300E0FF90028AE0F8A3E0F9A3E0FAA3E0FBF0
:1023A300EF2BFFEE3AFEED39FDEC38FC900286127E
:1023B3005339900282E0F8A3E0F9A3E0FAA3E0FB2B
:1023C300C000C001C002C00390027EE0FCA3E0FD98
:1023D300A3E0FEA3E0FF12523190028AE0F8A3E0EB
:1023E300F9A3E0FAA3E0FBEF5BFFEE5AFEED59FD24
:1023F300EC58FCC004C005C006C00790027EE0FC98
:10240300A3E0FDA3E0FEA3E0FF900286E0F8A3E0D3
:10241300F9A3E0FAA3E0FBEB5FFFEA5EFEE95DFDF3
:10242300E85CFCD003D002D001D000EF4BFFEE4AB2
:10243300FEED49FDEC48FC9002AEE0F8A3E0F9A301
:10244300E0FAA3E0FBEF2BFFEE3AFEED39FDEC38AB
:10245300FCEF24EDFFEE3414FEED345AFDEC34456D
:10246300FCD003D002D001D000EB2FFFEA3EFEE9FF
:102473003DFDE83CFC900282125339900282E0FC5D
:10248300A3E0FDA3E0FEA3E0FF7814125278C0049A
:10249300C005C006C007900282E0FCA3E0FDA3E0F4
:1024A300FEA3E0FF780C125265A804A905AA06ABA7
:1024B30007D007D006D005D004EB4FFFEA4EFEE964
:1024C3004DFDE84CFC900282125339900282E0FCED
:1024D300A3E0FDA3E0FEA3E0FF900286E0F8A3E003
:1024E300F9A3E0FAA3E0FBEF2BFFEE3AFEED39FD93
:1024F300EC38FC90028212533990027EE0F8A3E09C
:10250300F9A3E0FAA3E0FBC000C001C002C003903E
:10251300028AE0FCA3E0FDA3E0FEA3E0FF12523138
:10252300900286E0F8A3E0F9A3E0FAA3E0FBEF5BF7
:10253300FFEE5AFEED59FDEC58FCC004C005C00681
:10254300C00790028AE0FCA3E0FDA3E0FEA3E0FF46
:10255300900282E0F8A3E0F9A3E0FAA3E0FBEB5FCB
:10256300FFEA5EFEE95DFDE85CFCD003D002D0012A
:10257300D000EF4BFFEE4AFEED49FDEC48FC900224
:10258300C2E0F8A3E0F9A3E0FAA3E0FBEF2BFFEE30
:102593003AFEED39FDEC38FCEF2405FFEE34E9FE9D
:1025A300ED34E3FDEC34A9FCD003D002D001D0001C
:1025B300EB2FFFEA3EFEE93DFDE83CFC90027E1274
:1025C300533990027EE0FCA3E0FDA3E0FEA3E0FF0D
:1025D3007805125278C004C005C006C00790027E79
:1025E300E0FCA3E0FDA3E0FEA3E0FF781B1252652D
:1025F300A804A905AA06AB07D007D006D005D004C6
:10260300EB4FFFEA4EFEE94DFDE84CFC90027E12D3
:10261300533990027EE0FCA3E0FDA3E0FEA3E0FFBC
:10262300900282E0F8A3E0F9A3E0FAA3E0FBEF2B2A
:10263300FFEE3AFEED39FDEC38FC90027E12533981
:1026430090028AE0F8A3E0F9A3E0FAA3E0FBC0005C
:10265300C001C002C003900286E0FCA3E0FDA3E03A
:10266300FEA3E0FF125231900282E0F8A3E0F9A347
:10267300E0FAA3E0FBEF5BFFEE5AFEED59FDEC58E9
:10268300FCC004C005C006C007900286E0FCA3E0BE
:10269300FDA3E0FEA3E0FF90027EE0F8A3E0F9A330
:1026A300E0FAA3E0FBEB5FFFEA5EFEE95DFDE85CB9
:1026B300FCD003D002D001D000EF4BFFEE4AFEED79
:1026C30049FDEC48FC900296E0F8A3E0F9A3E0FA98
:1026D300A3E0FBEF2BFFEE3AFEED39FDEC38FCEF08
:1026E30024F8FFEE34A3FEED34EFFDEC34FCFCD014
:1026F30003D002D001D000EB2FFFEA3EFEE93DFDFF
:10270300E83CFC90028A12533990028AE0FCA3E071
:10271300FDA3E0FEA3E0FF7809125278C004C005D0
:10272300C006C00790028AE0FCA3E0FDA3E0FEA37D
:10273300E0FF7817125265A804A905AA06AB07D0D3
:1027430007D006D005D004EB4FFFEA4EFEE94DFD5E
:10275300E84CFC90028A12533990028AE0FCA3E011
:10276300FDA3E0FEA3E0FF90027EE0F8A3E0F9A35F
:10277300E0FAA3E0FBEF2BFFEE3AFEED39FDEC3878
:10278300FC90028A125339900286E0F8A3E0F9A381
:10279300E0FAA3E0FBC000C001C002C003900282C4
:1027A300E0FCA3E0FDA3E0FEA3E0FF1252319002A0
:1027B3007EE0F8A3E0F9A3E0FAA3E0FBEF5BFFEE12
:1027C3005AFEED59FDEC58FCC004C005C006C00715
:1027D300900282E0FCA3E0FDA3E0FEA3E0FF9002F1
:1027E3008AE0F8A3E0F9A3E0FAA3E0FBEB5FFFEADA
:1027F3005EFEE95DFDE85CFCD003D002D001D000B1
:10280300EF4BFFEE4AFEED49FDEC48FC9002AAE0D7
:10281300F8A3E0F9A3E0FAA3E0FBEF2BFFEE3AFE07
:10282300ED39FDEC38FCEF24D9FFEE3402FEED3434
:102833006FFDEC3467FCD003D002D001D000EB2F46
:10284300FFEA3EFEE93DFDE83CFC90028612533967
:10285300900286E0FCA3E0FDA3E0FEA3E0FF780E78
:10286300125278C004C005C006C007900286E0FC7F
:10287300A3E0FDA3E0FEA3E0FF7812125265A804D3
:10288300A905AA06AB07D007D006D005D004EB4FA5
:10289300FFEA4EFEE94DFDE84CFC900286125339E7
:1028A300900286E0FCA3E0FDA3E0FEA3E0FF90021C
:1028B3008AE0F8A3E0F9A3E0FAA3E0FBEF2BFFEE35
:1028C3003AFEED39FDEC38FC900286125339900242
:1028D30082E0F8A3E0F9A3E0FAA3E0FBC000C001A3
:1028E300C002C00390027EE0FCA3E0FDA3E0FEA3D0
:1028F300E0FF12523190028AE0F8A3E0F9A3E0FA74
:10290300A3E0FBEF5BFFEE5AFEED59FDEC58FCC074
:1029130004C005C006C00790027EE0FCA3E0FDA34F
:10292300E0FEA3E0FF900286E0F8A3E0F9A3E0FA5B
:10293300A3E0FBEB5FFFEA5EFEE95DFDE85CFCD034
:1029430003D002D001D000EF4BFFEE4AFEED49FD6C
:10295300EC48FC9002BEE0F8A3E0F9A3E0FAA3E0A0
:10296300FBEF2BFFEE3AFEED39FDEC38FCEF248A4A
:10297300FFEE344CFEED342AFDEC348DFCD003D055
:1029830002D001D000EB2FFFEA3EFEE93DFDE83C1B
:10299300FC900282125339900282E0FCA3E0FDA373
:1029A300E0FEA3E0FF7814125278C004C005C0060D
:1029B300C007900282E0FCA3E0FDA3E0FEA3E0FFDA
:1029C300780C125265A804A905AA06AB07D007D054
:1029D30006D005D004EB4FFFEA4EFEE94DFDE84C6F
:1029E300FC900282125339900282E0FCA3E0FDA323
:1029F300E0FEA3E0FF900286E0F8A3E0F9A3E0FA8B
:102A0300A3E0FBEF2BFFEE3AFEED39FDEC38FC9033
:102A1300028212533990027EE0F8A3E0F9A3E0FAB0
:102A2300A3E0FBC000C001C002C003900286E0FC2B
:102A3300A3E0FDA3E0FEA3E0FF900282E0F8A3E0A1
:102A4300F9A3E0FAA3E0FBEB6FFFEA6EFEE96DFD8D
:102A5300E86CFC90028AE0F8A3E0F9A3E0FAA3E0B3
:102A6300FBEF6BFFEE6AFEED69FDEC68FC9002A2E2
:102A7300E0F8A3E0F9A3E0FAA3E0FBEF2BFFEE3AC3
:102A8300FEED39FDEC38FCEF2442FFEE3439FEED68
:102A930034FAFDEC34FFFCD003D002D001D000EBBC
:102AA3002FFFEA3EFEE93DFDE83CFC90027E125317
:102AB3003990027EE0FCA3E0FDA3E0FEA3E0FF78F3
:102AC30004125278C004C005C006C00790027EE01D
:102AD300FCA3E0FDA3E0FEA3E0FF781C125265A86F
:102AE30004A905AA06AB07D007D006D005D004EB8E
:102AF3004FFFEA4EFEE94DFDE84CFC90027E125377
:102B03003990027EE0FCA3E0FDA3E0FEA3E0FF908A
:102B13000282E0F8A3E0F9A3E0FAA3E0FBEF2BFFC6
:102B2300EE3AFEED39FDEC38FC90027E12533990FB
:102B3300028AE0F8A3E0F9A3E0FAA3E0FBC000C037
:102B430001C002C003900282E0FCA3E0FDA3E0FE0B
:102B5300A3E0FF90027EE0F8A3E0F9A3E0FAA3E08C
:102B6300FBEB6FFFEA6EFEE96DFDE86CFC900286FD
:102B7300E0F8A3E0F9A3E0FAA3E0FBEF6BFFEE6A52
:102B8300FEED69FDEC68FC9002AEE0F8A3E0F9A36A
:102B9300E0FAA3E0FBEF2BFFEE3AFEED39FDEC3854
:102BA300FCEF2481FFEE34F6FEED3471FDEC348747
:102BB300FCD003D002D001D000EB2FFFEA3EFEE9A8
:102BC3003DFDE83CFC90028A12533990028AE0FCF6
:102BD300A3E0FDA3E0FEA3E0FF780B125278C0044C
:102BE300C005C006C00790028AE0FCA3E0FDA3E095
:102BF300FEA3E0FF7815125265A804A905AA06AB47
:102C030007D007D006D005D004EB4FFFEA4EFEE90C
:102C13004DFDE84CFC90028A12533990028AE0FC85
:102C2300A3E0FDA3E0FEA3E0FF90027EE0F8A3E0B3
:102C3300F9A3E0FAA3E0FBEF2BFFEE3AFEED39FD3B
:102C4300EC38FC90028A125339900286E0F8A3E034
:102C5300F9A3E0FAA3E0FBC000C001C002C00390E7
:102C6300027EE0FCA3E0FDA3E0FEA3E0FF90028A66
:102C7300E0F8A3E0F9A3E0FAA3E0FBEB6FFFEA6E51
:102C8300FEE96DFDE86CFC900282E0F8A3E0F9A395
:102C9300E0FAA3E0FBEF6BFFEE6AFEED69FDEC6883
:102CA300FC9002BAE0F8A3E0F9A3E0FAA3E0FBEF9B
:102CB3002BFFEE3AFEED39FDEC38FCEF2422FFEE5C
:102CC3003461FEED349DFDEC346DFCD003D002D0B5
:102CD30001D000EB2FFFEA3EFEE93DFDE83CFC900E
:102CE3000286125339900286E0FCA3E0FDA3E0FEC6
:102CF300A3E0FF7810125278C004C005C006C007D5
:102D0300900286E0FCA3E0FDA3E0FEA3E0FF7810C1
:102D1300125265A804A905AA06AB07D007D006D0AE
:102D230005D004EB4FFFEA4EFEE94DFDE84CFC9065
:102D33000286125339900286E0FCA3E0FDA3E0FE75
:102D4300A3E0FF90028AE0F8A3E0F9A3E0FAA3E08E
:102D5300FBEF2BFFEE3AFEED39FDEC38FC900286DB
:102D6300125339900282E0F8A3E0F9A3E0FAA3E05A
:102D7300FBC000C001C002C00390028AE0FCA3E0D4
:102D8300FDA3E0FEA3E0FF900286E0F8A3E0F9A331
:102D9300E0FAA3E0FBEB6FFFEA6EFEE96DFDE86C82
:102DA300FC90027EE0F8A3E0F9A3E0FAA3E0FBEFD6
:102DB3006BFFEE6AFEED69FDEC68FC9002C6E0F87D
:102DC300A3E0F9A3E0FAA3E0FBEF2BFFEE3AFEED5D
:102DD30039FDEC38FCEF240CFFEE3438FEED34E51E
:102DE300FDEC34FDFCD003D002D001D000EB2FFF6B
:102DF300EA3EFEE93DFDE83CFC9002821253399025
:102E03000282E0FCA3E0FDA3E0FEA3E0FF7817123B
:102E13005278C004C005C006C007900282E0FCA33C
:102E2300E0FDA3E0FEA3E0FF7809125265A804A920
:102E330005AA06AB07D007D006D005D004EB4FFF99
:102E4300EA4EFEE94DFDE84CFC90028212533990A4
:102E53000282E0FCA3E0FDA3E0FEA3E0FF90028674
:102E6300E0F8A3E0F9A3E0FAA3E0FBEF2BFFEE3ACF
:102E7300FEED39FDEC38FC90028212533990027E4C
:102E8300E0F8A3E0F9A3E0FAA3E0FBC000C001C0AF
:102E930002C003900286E0FCA3E0FDA3E0FEA3E0F2
:102EA300FF900282E0F8A3E0F9A3E0FAA3E0FBEBD2
:102EB3006FFFEA6EFEE96DFDE86CFC90028AE0F8B4
:102EC300A3E0F9A3E0FAA3E0FBEF6BFFEE6AFEEDEC
:102ED30069FDEC68FC900292E0F8A3E0F9A3E0FA44
:102EE300A3E0FBEF2BFFEE3AFEED39FDEC38FCEFF0
:102EF3002444FFEE34EAFEED34BEFDEC34A4FCD0F2
:102F030003D002D001D000EB2FFFEA3EFEE93DFDE6
:102F1300E83CFC90027E12533990027EE0FCA3E071
:102F2300FDA3E0FEA3E0FF7804125278C004C005BD
:102F3300C006C00790027EE0FCA3E0FDA3E0FEA371
:102F4300E0FF781C125265A804A905AA06AB07D0B6
:102F530007D006D005D004EB4FFFEA4EFEE94DFD46
:102F6300E84CFC90027E12533990027EE0FCA3E011
:102F7300FDA3E0FEA3E0FF900282E0F8A3E0F9A343
:102F8300E0FAA3E0FBEF2BFFEE3AFEED39FDEC3860
:102F9300FC90027E12533990028AE0F8A3E0F9A371
:102FA300E0FAA3E0FBC000C001C002C003900282AC
:102FB300E0FCA3E0FDA3E0FEA3E0FF90027EE0F8C7
:102FC300A3E0F9A3E0FAA3E0FBEB6FFFEA6EFEE9EF
:102FD3006DFDE86CFC900286E0F8A3E0F9A3E0FA4B
:102FE300A3E0FBEF6BFFEE6AFEED69FDEC68FC907E
:102FF300029EE0F8A3E0F9A3E0FAA3E0FBEF2BFFC6
:10300300EE3AFEED39FDEC38FCEF24A9FFEE34CFA8
:10301300FEED34DEFDEC344BFCD003D002D001D006
:1030230000EB2FFFEA3EFEE93DFDE83CFC90028AFF
:1030330012533990028AE0FCA3E0FDA3E0FEA3E073
:10304300FF780B125278C004C005C006C007900277
:103053008AE0FCA3E0FDA3E0FEA3E0FF7815125293
:1030630065A804A905AA06AB07D007D006D005D0EA
:1030730004EB4FFFEA4EFEE94DFDE84CFC90028A5B
:1030830012533990028AE0FCA3E0FDA3E0FEA3E023
:10309300FF90027EE0F8A3E0F9A3E0FAA3E0FBEFE0
:1030A3002BFFEE3AFEED39FDEC38FC90028A125309
:1030B30039900286E0F8A3E0F9A3E0FAA3E0FBC0AD
:1030C30000C001C002C00390027EE0FCA3E0FDA3A8
:1030D300E0FEA3E0FF90028AE0F8A3E0F9A3E0FAA0
:1030E300A3E0FBEB6FFFEA6EFEE96DFDE86CFC907D
:1030F3000282E0F8A3E0F9A3E0FAA3E0FBEF6BFFA1
:10310300EE6AFEED69FDEC68FC9002AAE0F8A3E02C
:10311300F9A3E0FAA3E0FBEF2BFFEE3AFEED39FD56
:10312300EC38FCEF2460FFEE344BFEED34BBFDECDA
:1031330034F6FCD003D002D001D000EB2FFFEA3EDF
:10314300FEE93DFDE83CFC9002861253399002866D
:10315300E0FCA3E0FDA3E0FEA3E0FF7810125278A9
:10316300C004C005C006C007900286E0FCA3E0FDD2
:10317300A3E0FEA3E0FF7810125265A804A905AAF4
:1031830006AB07D007D006D005D004EB4FFFEA4EBD
:10319300FEE94DFDE84CFC900286125339900286FD
:1031A300E0FCA3E0FDA3E0FEA3E0FF90028AE0F8C9
:1031B300A3E0F9A3E0FAA3E0FBEF2BFFEE3AFEED69
:1031C30039FDEC38FC900286125339900282E0F804
:1031D300A3E0F9A3E0FAA3E0FBC000C001C002C072
:1031E3000390028AE0FCA3E0FDA3E0FEA3E0FF90CE
:1031F3000286E0F8A3E0F9A3E0FAA3E0FBEB6FFF9C
:10320300EA6EFEE96DFDE86CFC90027EE0F8A3E057
:10321300F9A3E0FAA3E0FBEF6BFFEE6AFEED69FDB5
:10322300EC68FC9002B6E0F8A3E0F9A3E0FAA3E0AF
:10323300FBEF2BFFEE3AFEED39FDEC38FCEF24708B
:10324300FFEE34BCFEED34BFFDEC34BEFCD003D046
:1032530002D001D000EB2FFFEA3EFEE93DFDE83C42
:10326300FC900282125339900282E0FCA3E0FDA39A
:10327300E0FEA3E0FF7817125278C004C005C00631
:10328300C007900282E0FCA3E0FDA3E0FEA3E0FF01
:103293007809125265A804A905AA06AB07D007D07E
:1032A30006D005D004EB4FFFEA4EFEE94DFDE84C96
:1032B300FC900282125339900282E0FCA3E0FDA34A
:1032C300E0FEA3E0FF900286E0F8A3E0F9A3E0FAB2
:1032D300A3E0FBEF2BFFEE3AFEED39FDEC38FC905B
:1032E300028212533990027EE0F8A3E0F9A3E0FAD8
:1032F300A3E0FBC000C001C002C003900286E0FC53
:10330300A3E0FDA3E0FEA3E0FF900282E0F8A3E0C8
:10331300F9A3E0FAA3E0FBEB6FFFEA6EFEE96DFDB4
:10332300E86CFC90028AE0F8A3E0F9A3E0FAA3E0DA
:10333300FBEF6BFFEE6AFEED69FDEC68FC9002C2E9
:10334300E0F8A3E0F9A3E0FAA3E0FBEF2BFFEE3AEA
:10335300FEED39FDEC38FCEF24C6FFEE347EFEEDC6
:10336300349BFDEC3428FCD003D002D001D000EB19
:103373002FFFEA3EFEE93DFDE83CFC90027E12533E
:103383003990027EE0FCA3E0FDA3E0FEA3E0FF781A
:1033930004125278C004C005C006C00790027EE044
:1033A300FCA3E0FDA3E0FEA3E0FF781C125265A896
:1033B30004A905AA06AB07D007D006D005D004EBB5
:1033C3004FFFEA4EFEE94DFDE84CFC90027E12539E
:1033D3003990027EE0FCA3E0FDA3E0FEA3E0FF90B2
:1033E3000282E0F8A3E0F9A3E0FAA3E0FBEF2BFFEE
:1033F300EE3AFEED39FDEC38FC90027E1253399023
:10340300028AE0F8A3E0F9A3E0FAA3E0FBC000C05E
:1034130001C002C003900282E0FCA3E0FDA3E0FE32
:10342300A3E0FF90027EE0F8A3E0F9A3E0FAA3E0B3
:10343300FBEB6FFFEA6EFEE96DFDE86CFC90028624
:10344300E0F8A3E0F9A3E0FAA3E0FBEF6BFFEE6A79
:10345300FEED69FDEC68FC90028EE0F8A3E0F9A3B1
:10346300E0FAA3E0FBEF2BFFEE3AFEED39FDEC387B
:10347300FCEF24FAFFEE3427FEED34A1FDEC34EA31
:10348300FCD003D002D001D000EB2FFFEA3EFEE9CF
:103493003DFDE83CFC90028A12533990028AE0FC1D
:1034A300A3E0FDA3E0FEA3E0FF780B125278C00473
:1034B300C005C006C00790028AE0FCA3E0FDA3E0BC
:1034C300FEA3E0FF7815125265A804A905AA06AB6E
:1034D30007D007D006D005D004EB4FFFEA4EFEE934
:1034E3004DFDE84CFC90028A12533990028AE0FCAD
:1034F300A3E0FDA3E0FEA3E0FF90027EE0F8A3E0DB
:10350300F9A3E0FAA3E0FBEF2BFFEE3AFEED39FD62
:10351300EC38FC90028A125339900286E0F8A3E05B
:10352300F9A3E0FAA3E0FBC000C001C002C003900E
:10353300027EE0FCA3E0FDA3E0FEA3E0FF90028A8D
:10354300E0F8A3E0F9A3E0FAA3E0FBEB6FFFEA6E78
:10355300FEE96DFDE86CFC900282E0F8A3E0F9A3BC
:10356300E0FAA3E0FBEF6BFFEE6AFEED69FDEC68AA
:10357300FC90029AE0F8A3E0F9A3E0FAA3E0FBEFE2
:103583002BFFEE3AFEED39FDEC38FCEF2485FFEE20
:103593003430FEED34EFFDEC34D4FCD003D002D054
:1035A30001D000EB2FFFEA3EFEE93DFDE83CFC9035
:1035B3000286125339900286E0FCA3E0FDA3E0FEED
:1035C300A3E0FF7810125278C004C005C006C007FC
:1035D300900286E0FCA3E0FDA3E0FEA3E0FF7810E9
:1035E300125265A804A905AA06AB07D007D006D0D6
:1035F30005D004EB4FFFEA4EFEE94DFDE84CFC908D
:103603000286125339900286E0FCA3E0FDA3E0FE9C
:10361300A3E0FF90028AE0F8A3E0F9A3E0FAA3E0B5
:10362300FBEF2BFFEE3AFEED39FDEC38FC90028602
:10363300125339900282E0F8A3E0F9A3E0FAA3E081
:10364300FBC000C001C002C00390028AE0FCA3E0FB
:10365300FDA3E0FEA3E0FF900286E0F8A3E0F9A358
:10366300E0FAA3E0FBEB6FFFEA6EFEE96DFDE86CA9
:10367300FC90027EE0F8A3E0F9A3E0FAA3E0FBEFFD
:103683006BFFEE6AFEED69FDEC68FC9002A6E0F8C4
:10369300A3E0F9A3E0FAA3E0FBEF2BFFEE3AFEED84
:1036A30039FDEC38FCEF2405FFEE341DFEED3488C4
:1036B300FDEC3404FCD003D002D001D000EB2FFF8B
:1036C300EA3EFEE93DFDE83CFC900282125339904C
:1036D3000282E0FCA3E0FDA3E0FEA3E0FF78171263
:1036E3005278C004C005C006C007900282E0FCA364
:1036F300E0FDA3E0FEA3E0FF7809125265A804A948
:1037030005AA06AB07D007D006D005D004EB4FFFC0
:10371300EA4EFEE94DFDE84CFC90028212533990CB
:103723000282E0FCA3E0FDA3E0FEA3E0FF9002869B
:10373300E0F8A3E0F9A3E0FAA3E0FBEF2BFFEE3AF6
:10374300FEED39FDEC38FC90028212533990027E73
:10375300E0F8A3E0F9A3E0FAA3E0FBC000C001C0D6
:1037630002C003900286E0FCA3E0FDA3E0FEA3E019
:10377300FF900282E0F8A3E0F9A3E0FAA3E0FBEBF9
:103783006FFFEA6EFEE96DFDE86CFC90028AE0F8DB
:10379300A3E0F9A3E0FAA3E0FBEF6BFFEE6AFEED13
:1037A30069FDEC68FC9002B2E0F8A3E0F9A3E0FA4B
:1037B300A3E0FBEF2BFFEE3AFEED39FDEC38FCEF17
:1037C3002439FFEE34D0FEED34D4FDEC34D9FCD0F3
:1037D30003D002D001D000EB2FFFEA3EFEE93DFD0E
:1037E300E83CFC90027E12533990027EE0FCA3E099
:1037F300FDA3E0FEA3E0FF7804125278C004C005E5
:10380300C006C00790027EE0FCA3E0FDA3E0FEA398
:10381300E0FF781C125265A804A905AA06AB07D0DD
:1038230007D006D005D004EB4FFFEA4EFEE94DFD6D
:10383300E84CFC90027E12533990027EE0FCA3E038
:10384300FDA3E0FEA3E0FF900282E0F8A3E0F9A36A
:10385300E0FAA3E0FBEF2BFFEE3AFEED39FDEC3887
:10386300FC90027E12533990028AE0F8A3E0F9A398
:10387300E0FAA3E0FBC000C001C002C003900282D3
:10388300E0FCA3E0FDA3E0FEA3E0FF90027EE0F8EE
:10389300A3E0F9A3E0FAA3E0FBEB6FFFEA6EFEE916
:1038A3006DFDE86CFC900286E0F8A3E0F9A3E0FA72
:1038B300A3E0FBEF6BFFEE6AFEED69FDEC68FC90A5
:1038C30002BEE0F8A3E0F9A3E0FAA3E0FBEF2BFFCD
:1038D300EE3AFEED39FDEC38FCEF24E5FFEE3499CA
:1038E300FEED34DBFDEC34E6FCD003D002D001D096
:1038F30000EB2FFFEA3EFEE93DFDE83CFC90028A27
:1039030012533990028AE0FCA3E0FDA3E0FEA3E09A
:10391300FF780B125278C004C005C006C00790029E
:103923008AE0FCA3E0FDA3E0FEA3E0FF78151252BA
:1039330065A804A905AA06AB07D007D006D005D011
:1039430004EB4FFFEA4EFEE94DFDE84CFC90028A82
:1039530012533990028AE0FCA3E0FDA3E0FEA3E04A
:10396300FF90027EE0F8A3E0F9A3E0FAA3E0FBEF07
:103973002BFFEE3AFEED39FDEC38FC90028A125330
:1039830039900286E0F8A3E0F9A3E0FAA3E0FBC0D4
:1039930000C001C002C00390027EE0FCA3E0FDA3CF
:1039A300E0FEA3E0FF90028AE0F8A3E0F9A3E0FAC7
:1039B300A3E0FBEB6FFFEA6EFEE96DFDE86CFC90A4
:1039C3000282E0F8A3E0F9A3E0FAA3E0FBEF6BFFC8
:1039D300EE6AFEED69FDEC68FC9002CAE0F8A3E034
:1039E300F9A3E0FAA3E0FBEF2BFFEE3AFEED39FD7E
:1039F300EC38FCEF24F8FFEE347CFEED34A2FDEC52
:103A0300341FFCD003D002D001D000EB2FFFEA3EDD
:103A1300FEE93DFDE83CFC90028612533990028694
:103A2300E0FCA3E0FDA3E0FEA3E0FF7810125278D0
:103A3300C004C005C006C007900286E0FCA3E0FDF9
:103A4300A3E0FEA3E0FF7810125265A804A905AA1B
:103A530006AB07D007D006D005D004EB4FFFEA4EE4
:103A6300FEE94DFDE84CFC90028612533990028624
:103A7300E0FCA3E0FDA3E0FEA3E0FF90028AE0F8F0
:103A8300A3E0F9A3E0FAA3E0FBEF2BFFEE3AFEED90
:103A930039FDEC38FC900286125339900282E0F82B
:103AA300A3E0F9A3E0FAA3E0FBC000C001C002C099
:103AB3000390028AE0FCA3E0FDA3E0FEA3E0FF90F5
:103AC3000286E0F8A3E0F9A3E0FAA3E0FBEB6FFFC3
:103AD300EA6EFEE96DFDE86CFC90027EE0F8A3E07F
:103AE300F9A3E0FAA3E0FBEF6BFFEE6AFEED69FDDD
:103AF300EC68FC900296E0F8A3E0F9A3E0FAA3E0F7
:103B0300FBEF2BFFEE3AFEED39FDEC38FCEF2465BD
:103B1300FFEE3456FEED34ACFDEC34C4FCD003D0E0
:103B230002D001D000EB2FFFEA3EFEE93DFDE83C69
:103B3300FC900282125339900282E0FCA3E0FDA3C1
:103B4300E0FEA3E0FF7817125278C004C005C00658
:103B5300C007900282E0FCA3E0FDA3E0FEA3E0FF28
:103B63007809125265A804A905AA06AB07D007D0A5
:103B730006D005D004EB4FFFEA4EFEE94DFDE84CBD
:103B8300FC900282125339900282E0FCA3E0FDA371
:103B9300E0FEA3E0FF900286E0F8A3E0F9A3E0FAD9
:103BA300A3E0FBEF2BFFEE3AFEED39FDEC38FC9082
:103BB300028212533990027EE0F8A3E0F9A3E0FAFF
:103BC300A3E0FBC000C001C002C00390028AE0FC76
:103BD300A3E0FDA3E0FEA3E0FF125231900282E0D6
:103BE300F8A3E0F9A3E0FAA3E0FBEF4BFFEE4AFEF4
:103BF300ED49FDEC48FC900286E0F8A3E0F9A3E070
:103C0300FAA3E0FBEF6BFFEE6AFEED69FDEC68FCE7
:103C130090028EE0F8A3E0F9A3E0FAA3E0FBEF2B18
:103C2300FFEE3AFEED39FDEC38FCEF2444FFEE34B1
:103C330022FEED3429FDEC34F4FCD003D002D00194
:103C4300D000EB2FFFEA3EFEE93DFDE83CFC90028D
:103C53007E12533990027EE0FCA3E0FDA3E0FEA3B5
:103C6300E0FF7806125278C004C005C006C0079072
:103C7300027EE0FCA3E0FDA3E0FEA3E0FF781A12BE
:103C83005265A804A905AA06AB07D007D006D0053C
:103C9300D004EB4FFFEA4EFEE94DFDE84CFC9002E9
:103CA3007E12533990027EE0FCA3E0FDA3E0FEA365
:103CB300E0FF900282E0F8A3E0F9A3E0FAA3E0FBBF
:103CC300EF2BFFEE3AFEED39FDEC38FC90027E124D
:103CD300533990028AE0F8A3E0F9A3E0FAA3E0FBEA
:103CE300C000C001C002C003900286E0FCA3E0FD57
:103CF300A3E0FEA3E0FF12523190027EE0F8A3E0BE
:103D0300F9A3E0FAA3E0FBEF4BFFEE4AFEED49FD1A
:103D1300EC48FC900282E0F8A3E0F9A3E0FAA3E008
:103D2300FBEF6BFFEE6AFEED69FDEC68FC9002AA07
:103D3300E0F8A3E0F9A3E0FAA3E0FBEF2BFFEE3AF0
:103D4300FEED39FDEC38FCEF2497FFEE34FFFEED7A
:103D5300342AFDEC3443FCD003D002D001D000EB75
:103D63002FFFEA3EFEE93DFDE83CFC90028A125338
:103D73003990028AE0FCA3E0FDA3E0FEA3E0FF7814
:103D83000A125278C004C005C006C00790028AE038
:103D9300FCA3E0FDA3E0FEA3E0FF7816125265A8A2
:103DA30004A905AA06AB07D007D006D005D004EBBB
:103DB3004FFFEA4EFEE94DFDE84CFC90028A125398
:103DC3003990028AE0FCA3E0FDA3E0FEA3E0FF90AC
:103DD300027EE0F8A3E0F9A3E0FAA3E0FBEF2BFFF8
:103DE300EE3AFEED39FDEC38FC90028A125339901D
:103DF3000286E0F8A3E0F9A3E0FAA3E0FBC000C069
:103E030001C002C003900282E0FCA3E0FDA3E0FE38
:103E1300A3E0FF12523190028AE0F8A3E0F9A3E095
:103E2300FAA3E0FBEF4BFFEE4AFEED49FDEC48FC45
:103E330090027EE0F8A3E0F9A3E0FAA3E0FBEF6BC6
:103E4300FFEE6AFEED69FDEC68FC9002C6E0F8A3A4
:103E5300E0F9A3E0FAA3E0FBEF2BFFEE3AFEED3926
:103E6300FDEC38FCEF24A7FFEE3423FEED3494FD84
:103E7300EC34ABFCD003D002D001D000EB2FFFEA2F
:103E83003EFEE93DFDE83CFC900286125339900268
:103E930086E0FCA3E0FDA3E0FEA3E0FF780F12524F
:103EA30078C004C005C006C007900286E0FCA3E00A
:103EB300FDA3E0FEA3E0FF7811125265A804A90553
:103EC300AA06AB07D007D006D005D004EB4FFFEA14
:103ED3004EFEE94DFDE84CFC9002861253399002E8
:103EE30086E0FCA3E0FDA3E0FEA3E0FF90028AE0EE
:103EF300F8A3E0F9A3E0FAA3E0FBEF2BFFEE3AFE11
:103F0300ED39FDEC38FC900286125339900282E0C1
:103F1300F8A3E0F9A3E0FAA3E0FBC000C001C002EC
:103F2300C00390027EE0FCA3E0FDA3E0FEA3E0FF5C
:103F3300125231900286E0F8A3E0F9A3E0FAA3E07D
:103F4300FBEF4BFFEE4AFEED49FDEC48FC90028A85
:103F5300E0F8A3E0F9A3E0FAA3E0FBEF6BFFEE6A5E
:103F6300FEED69FDEC68FC9002A2E0F8A3E0F9A382
:103F7300E0FAA3E0FBEF2BFFEE3AFEED39FDEC3860
:103F8300FCEF2439FFEE34A0FEED3493FDEC34FC5A
:103F9300FCD003D002D001D000EB2FFFEA3EFEE9B4
:103FA3003DFDE83CFC900282125339900282E0FC12
:103FB300A3E0FDA3E0FEA3E0FF7815125278C0044E
:103FC300C005C006C007900282E0FCA3E0FDA3E0A9
:103FD300FEA3E0FF780B125265A804A905AA06AB5D
:103FE30007D007D006D005D004EB4FFFEA4EFEE919
:103FF3004DFDE84CFC900282125339900282E0FCA2
:10400300A3E0FDA3E0FEA3E0FF900286E0F8A3E0B7
:10401300F9A3E0FAA3E0FBEF2BFFEE3AFEED39FD47
:10402300EC38FC90028212533990027EE0F8A3E050
:10403300F9A3E0FAA3E0FBC000C001C002C00390F3
:10404300028AE0FCA3E0FDA3E0FEA3E0FF125231ED
:10405300900282E0F8A3E0F9A3E0FAA3E0FBEF4BC0
:10406300FFEE4AFEED49FDEC48FC900286E0F8A322
:10407300E0F9A3E0FAA3E0FBEF6BFFEE6AFEED6964
:10408300FDEC68FC9002BEE0F8A3E0F9A3E0FAA31C
:10409300E0FBEF2BFFEE3AFEED39FDEC38FCEF24AD
:1040A300C3FFEE3459FEED345BFDEC3465FCD00305
:1040B300D002D001D000EB2FFFEA3EFEE93DFDE840
:1040C3003CFC90027E12533990027EE0FCA3E0FD9B
:1040D300A3E0FEA3E0FF7806125278C004C005C037
:1040E30006C00790027EE0FCA3E0FDA3E0FEA3E090
:1040F300FF781A125265A804A905AA06AB07D007D0
:10410300D006D005D004EB4FFFEA4EFEE94DFDE8A3
:104113004CFC90027E12533990027EE0FCA3E0FD3A
:10412300A3E0FEA3E0FF900282E0F8A3E0F9A3E09E
:10413300FAA3E0FBEF2BFFEE3AFEED39FDEC38FC82
:1041430090027E12533990028AE0F8A3E0F9A3E0CB
:10415300FAA3E0FBC000C001C002C003900286E0E6
:10416300FCA3E0FDA3E0FEA3E0FF12523190027E28
:10417300E0F8A3E0F9A3E0FAA3E0FBEF4BFFEE4A7C
:10418300FEED49FDEC48FC900282E0F8A3E0F9A3C0
:10419300E0FAA3E0FBEF6BFFEE6AFEED69FDEC686E
:1041A300FC90029AE0F8A3E0F9A3E0FAA3E0FBEFA6
:1041B3002BFFEE3AFEED39FDEC38FCEF2492FFEED7
:1041C30034CCFEED340CFDEC348FFCD003D002D0A4
:1041D30001D000EB2FFFEA3EFEE93DFDE83CFC90F9
:1041E300028A12533990028AE0FCA3E0FDA3E0FEA9
:1041F300A3E0FF780A125278C004C005C006C007C6
:1042030090028AE0FCA3E0FDA3E0FEA3E0FF7816A2
:10421300125265A804A905AA06AB07D007D006D099
:1042230005D004EB4FFFEA4EFEE94DFDE84CFC9050
:10423300028A12533990028AE0FCA3E0FDA3E0FE58
:10424300A3E0FF90027EE0F8A3E0F9A3E0FAA3E085
:10425300FBEF2BFFEE3AFEED39FDEC38FC90028AC2
:10426300125339900286E0F8A3E0F9A3E0FAA3E041
:10427300FBC000C001C002C003900282E0FCA3E0C7
:10428300FDA3E0FEA3E0FF12523190028AE0F8A3FF
:10429300E0F9A3E0FAA3E0FBEF4BFFEE4AFEED49A2
:1042A300FDEC48FC90027EE0F8A3E0F9A3E0FAA35A
:1042B300E0FBEF6BFFEE6AFEED69FDEC68FC90023C
:1042C300B6E0F8A3E0F9A3E0FAA3E0FBEF2BFFEEDF
:1042D3003AFEED39FDEC38FCEF247DFFEE34F4FEBD
:1042E300ED34EFFDEC34FFFCD003D002D001D0005D
:1042F300EB2FFFEA3EFEE93DFDE83CFC900286120F
:104303005339900286E0FCA3E0FDA3E0FEA3E0FFA7
:10431300780F125278C004C005C006C00790028609
:10432300E0FCA3E0FDA3E0FEA3E0FF7811125265D9
:10433300A804A905AA06AB07D007D006D005D00468
:10434300EB4FFFEA4EFEE94DFDE84CFC900286126E
:104353005339900286E0FCA3E0FDA3E0FEA3E0FF57
:1043630090028AE0F8A3E0F9A3E0FAA3E0FBEF2BC5
:10437300FFEE3AFEED39FDEC38FC9002861253391C
:10438300900282E0F8A3E0F9A3E0FAA3E0FBC00007
:10439300C001C002C00390027EE0FCA3E0FDA3E0E5
:1043A300FEA3E0FF125231900286E0F8A3E0F9A3E6
:1043B300E0FAA3E0FBEF4BFFEE4AFEED49FDEC48CC
:1043C300FC90028AE0F8A3E0F9A3E0FAA3E0FBEF94
:1043D3006BFFEE6AFEED69FDEC68FC900292E0F87B
:1043E300A3E0F9A3E0FAA3E0FBEF2BFFEE3AFEED27
:1043F30039FDEC38FCEF24D1FFEE345DFEED34845F
:10440300FDEC3485FCD003D002D001D000EB2FFFAC
:10441300EA3EFEE93DFDE83CFC90028212533990EE
:104423000282E0FCA3E0FDA3E0FEA3E0FF78151207
:104433005278C004C005C006C007900282E0FCA306
:10444300E0FDA3E0FEA3E0FF780B125265A804A9E8
:1044530005AA06AB07D007D006D005D004EB4FFF63
:10446300EA4EFEE94DFDE84CFC900282125339906E
:104473000282E0FCA3E0FDA3E0FEA3E0FF9002863E
:10448300E0F8A3E0F9A3E0FAA3E0FBEF2BFFEE3A99
:10449300FEED39FDEC38FC90028212533990027E16
:1044A300E0F8A3E0F9A3E0FAA3E0FBC000C001C079
:1044B30002C00390028AE0FCA3E0FDA3E0FEA3E0B8
:1044C300FF125231900282E0F8A3E0F9A3E0FAA3CD
:1044D300E0FBEF4BFFEE4AFEED49FDEC48FC90029A
:1044E30086E0F8A3E0F9A3E0FAA3E0FBEF6BFFEEAD
:1044F3006AFEED69FDEC68FC9002AEE0F8A3E0F91A
:10450300A3E0FAA3E0FBEF2BFFEE3AFEED39FDEC5F
:1045130038FCEF244FFFEE347EFEED34A8FDEC347F
:104523006FFCD003D002D001D000EB2FFFEA3EFE98
:10453300E93DFDE83CFC90027E12533990027EE097
:10454300FCA3E0FDA3E0FEA3E0FF7806125278C0CF
:1045530004C005C006C00790027EE0FCA3E0FDA3F3
:10456300E0FEA3E0FF781A125265A804A905AA0683
:10457300AB07D007D006D005D004EB4FFFEA4EFEC1
:10458300E94DFDE84CFC90027E12533990027EE027
:10459300FCA3E0FDA3E0FEA3E0FF900282E0F8A30A
:1045A300E0F9A3E0FAA3E0FBEF2BFFEE3AFEED39CF
:1045B300FDEC38FC90027E12533990028AE0F8A396
:1045C300E0F9A3E0FAA3E0FBC000C001C002C0030E
:1045D300900286E0FCA3E0FDA3E0FEA3E0FF1252FD
:1045E3003190027EE0F8A3E0F9A3E0FAA3E0FBEF49
:1045F3004BFFEE4AFEED49FDEC48FC900282E0F8E9
:10460300A3E0F9A3E0FAA3E0FBEF6BFFEE6AFEED94
:1046130069FDEC68FC9002CAE0F8A3E0F9A3E0FAB4
:10462300A3E0FBEF2BFFEE3AFEED39FDEC38FCEF98
:1046330024E0FFEE34E6FEED342CFDEC34FEFCD03A
:1046430003D002D001D000EB2FFFEA3EFEE93DFD8F
:10465300E83CFC90028A12533990028AE0FCA3E002
:10466300FDA3E0FEA3E0FF780A125278C004C00560
:10467300C006C00790028AE0FCA3E0FDA3E0FEA30E
:10468300E0FF7816125265A804A905AA06AB07D065
:1046930007D006D005D004EB4FFFEA4EFEE94DFDEF
:1046A300E84CFC90028A12533990028AE0FCA3E0A2
:1046B300FDA3E0FEA3E0FF90027EE0F8A3E0F9A3F0
:1046C300E0FAA3E0FBEF2BFFEE3AFEED39FDEC3809
:1046D300FC90028A125339900286E0F8A3E0F9A312
:1046E300E0FAA3E0FBC000C001C002C00390028255
:1046F300E0FCA3E0FDA3E0FEA3E0FF125231900231
:104703008AE0F8A3E0F9A3E0FAA3E0FBEF4BFFEEA6
:104713004AFEED49FDEC48FC90027EE0F8A3E0F987
:10472300A3E0FAA3E0FBEF6BFFEE6AFEED69FDEC9D
:1047330068FC9002A6E0F8A3E0F9A3E0FAA3E0FB8B
:10474300EF2BFFEE3AFEED39FDEC38FCEF2414FFBE
:10475300EE3443FEED3401FDEC34A3FCD003D00270
:10476300D001D000EB2FFFEA3EFEE93DFDE83CFC23
:10477300900286125339900286E0FCA3E0FDA3E089
:10478300FEA3E0FF780F125278C004C005C006C034
:1047930007900286E0FCA3E0FDA3E0FEA3E0FF7820
:1047A30011125265A804A905AA06AB07D007D006C3
:1047B300D005D004EB4FFFEA4EFEE94DFDE84CFC7B
:1047C300900286125339900286E0FCA3E0FDA3E039
:1047D300FEA3E0FF90028AE0F8A3E0F9A3E0FAA3C6
:1047E300E0FBEF2BFFEE3AFEED39FDEC38FC9002D7
:1047F30086125339900282E0F8A3E0F9A3E0FAA30A
:10480300E0FBC000C001C002C00390027EE0FCA335
:10481300E0FDA3E0FEA3E0FF125231900286E0F830
:10482300A3E0F9A3E0FAA3E0FBEF4BFFEE4AFEEDB2
:1048330049FDEC48FC90028AE0F8A3E0F9A3E0FA12
:10484300A3E0FBEF6BFFEE6AFEED69FDEC68FC9005
:1048530002C2E0F8A3E0F9A3E0FAA3E0FBEF2BFF29
:10486300EE3AFEED39FDEC38FCEF24A1FFEE3411F6
:10487300FEED3408FDEC344EFCD003D002D001D061
:1048830000EB2FFFEA3EFEE93DFDE83CFC9002828F
:10489300125339900282E0FCA3E0FDA3E0FEA3E003
:1048A300FF7815125278C004C005C006C0079002F5
:1048B30082E0FCA3E0FDA3E0FEA3E0FF780B12522D
:1048C30065A804A905AA06AB07D007D006D005D072
:1048D30004EB4FFFEA4EFEE94DFDE84CFC900282EB
:1048E300125339900282E0FCA3E0FDA3E0FEA3E0B3
:1048F300FF900286E0F8A3E0F9A3E0FAA3E0FBEF60
:104903002BFFEE3AFEED39FDEC38FC900282125398
:104913003990027EE0F8A3E0F9A3E0FAA3E0FBC03C
:1049230000C001C002C00390028AE0FCA3E0FDA323
:10493300E0FEA3E0FF125231900282E0F8A3E0F917
:10494300A3E0FAA3E0FBEF4BFFEE4AFEED49FDECDB
:1049530048FC900286E0F8A3E0F9A3E0FAA3E0FBA9
:10496300EF6BFFEE6AFEED69FDEC68FC90029EE0E2
:10497300F8A3E0F9A3E0FAA3E0FBEF2BFFEE3AFE86
:10498300ED39FDEC38FCEF2482FFEE347EFEED348E
:1049930053FDEC34F7FCD003D002D001D000EB2F51
:1049A300FFEA3EFEE93DFDE83CFC90027E125339EE
:1049B30090027EE0FCA3E0FDA3E0FEA3E0FF780607
:1049C300125278C004C005C006C00790027EE0FC06
:1049D300A3E0FDA3E0FEA3E0FF781A125265A8044A
:1049E300A905AA06AB07D007D006D005D004EB4F24
:1049F300FFEA4EFEE94DFDE84CFC90027E1253396E
:104A030090027EE0FCA3E0FDA3E0FEA3E0FF9002A2
:104A130082E0F8A3E0F9A3E0FAA3E0FBEF2BFFEEBB
:104A23003AFEED39FDEC38FC90027E1253399002C8
:104A33008AE0F8A3E0F9A3E0FAA3E0FBC000C00119
:104A4300C002C003900286E0FCA3E0FDA3E0FEA346
:104A5300E0FF12523190027EE0F8A3E0F9A3E0FAFE
:104A6300A3E0FBEF4BFFEE4AFEED49FDEC48FC9063
:104A73000282E0F8A3E0F9A3E0FAA3E0FBEF6BFF07
:104A8300EE6AFEED69FDEC68FC9002BAE0F8A3E083
:104A9300F9A3E0FAA3E0FBEF2BFFEE3AFEED39FDBD
:104AA300EC38FCEF2435FFEE34F2FEED343AFDEC46
:104AB30034BDFCD003D002D001D000EB2FFFEA3E7F
:104AC300FEE93DFDE83CFC90028A12533990028ACC
:104AD300E0FCA3E0FDA3E0FEA3E0FF780A12527816
:104AE300C004C005C006C00790028AE0FCA3E0FD35
:104AF300A3E0FEA3E0FF7816125265A804A905AA55
:104B030006AB07D007D006D005D004EB4FFFEA4E23
:104B1300FEE94DFDE84CFC90028A12533990028A5B
:104B2300E0FCA3E0FDA3E0FEA3E0FF90027EE0F83B
:104B3300A3E0F9A3E0FAA3E0FBEF2BFFEE3AFEEDCF
:104B430039FDEC38FC90028A125339900286E0F862
:104B5300A3E0F9A3E0FAA3E0FBC000C001C002C0D8
:104B630003900282E0FCA3E0FDA3E0FEA3E0FF12BA
:104B7300523190028AE0F8A3E0F9A3E0FAA3E0FB44
:104B8300EF4BFFEE4AFEED49FDEC48FC90027EE060
:104B9300F8A3E0F9A3E0FAA3E0FBEF6BFFEE6AFEF4
:104BA300ED69FDEC68FC900296E0F8A3E0F9A3E060
:104BB300FAA3E0FBEF2BFFEE3AFEED39FDEC38FCF8
:104BC300EF24BBFFEE34D2FEED34D7FDEC342AFCE8
:104BD300D003D002D001D000EB2FFFEA3EFEE93D27
:104BE300FDE83CFC900286125339900286E0FCA358
:104BF300E0FDA3E0FEA3E0FF780F125278C004C0EB
:104C030005C006C007900286E0FCA3E0FDA3E0FE1A
:104C1300A3E0FF7811125265A804A905AA06AB0701
:104C2300D007D006D005D004EB4FFFEA4EFEE94D86
:104C3300FDE84CFC900286125339900286E0FCA3F7
:104C4300E0FDA3E0FEA3E0FF90028AE0F8A3E0F911
:104C5300A3E0FAA3E0FBEF2BFFEE3AFEED39FDEC08
:104C630038FC900286125339900282E0F8A3E0F9EF
:104C7300A3E0FAA3E0FBC000C001C002C00390029E
:104C83007EE0FCA3E0FDA3E0FEA3E0FF125231901F
:104C93000286E0F8A3E0F9A3E0FAA3E0FBEF4BFF01
:104CA300EE4AFEED49FDEC48FC90028AE0F8A3E0F1
:104CB300F9A3E0FAA3E0FBEF6BFFEE6AFEED69FDFB
:104CC300EC68FC9002B2E0F8A3E0F9A3E0FAA3E0F9
:104CD300FBEF2BFFEE3AFEED39FDEC38FCEF2491B0
:104CE300FFEE34D3FEED3486FDEC34EBFCD003D081
:104CF30002D001D000EB2FFFEA3EFEE93DFDE83C88
:104D0300FC900282125339900282E0FCA3E0FDA3DF
:104D1300E0FEA3E0FF7815125278C004C005C00678
:104D2300C007900282E0FCA3E0FDA3E0FEA3E0FF46
:104D3300780B125265A804A905AA06AB07D007D0C1
:104D430006D005D004EB4FFFEA4EFEE94DFDE84CDB
:104D5300FC900282125339900282E0FCA3E0FDA38F
:104D6300E0FEA3E0FF900286E0F8A3E0F9A3E0FAF7
:104D7300A3E0FBEF2BFFEE3AFEED39FDEC38FC90A0
:104D83000282125339900278E0FBA3E0FAA3E0F920
:104D9300C003C002C00112528B90027EE0F8A3E070
:104DA300F9A3E0FAA3E0FBEF2BFFEE3AFEED39FDAA
:104DB300EC38FCD001D002D0031252DB900278E031
:104DC300FBA3E0FAA3E0F9E92404F9EA3400FAC00A
:104DD30003C002C00112528B900282E0F8A3E0F9F3
:104DE300A3E0FAA3E0FBEF2BFFEE3AFEED39FDEC77
:104DF30038FCD001D002D0031252DB900278E0FBE2
:104E0300A3E0FAA3E0F9E92408F9EA3400FAC003BD
:104E1300C002C00112528B900286E0F8A3E0F9A30E
:104E2300E0FAA3E0FBEF2BFFEE3AFEED39FDEC38A1
:104E3300FCD001D002D0031252DB900278E0FBA336
:104E4300E0FAA3E0F9E9240CF9EA3400FAC003C05C
:104E530002C00112528B90028AE0F8A3E0F9A3E0AA
:104E6300FAA3E0FBEF2BFFEE3AFEED39FDEC38FC45
:104E7300D001D002D0031252DB22E709F608DFFA91
:104E83008046E709F208DFFA803E88828C83E709CF
:104E9300F0A3DFFA8032E309F608DFFA8078E3094A
:104EA300F208DFFA807088828C83E309F0A3DFFACB
:104EB300806489828A83E0A3F608DFFA80588982B6
:104EC3008A83E0A3F208DFFA804C80D280FA80C69E
:104ED30080D4806980F28033801080A680EA809A33
:104EE30080A880DA80E280CA803389828A83ECFAE0
:104EF300E493A3C8C582C8CCC583CCF0A3C8C5823C
:104F0300C8CCC583CCDFE9DEE7800D89828A83E4E0
:104F130093A3F608DFF9ECFAA9F0EDFB2289828A64
:104F230083ECFAE0A3C8C582C8CCC583CCF0A3C880
:104F3300C582C8CCC583CCDFEADEE880DB89828A00
:104F430083E493A3F208DFF980CC88F0EF60010ECD
:104F53004E60C388F0ED2402B4040050B9F582EB2F
:104F63002402B4040050AF2323458223904ECD7313
:104F7300BB010689828A83E0225002E722BBFE023C
:104F8300E32289828A83E49322BB010CE58229F51B
:104F930082E5833AF583E0225006E92582F8E6228A
:104FA300BBFE06E92582F8E222E58229F582E58344
:104FB3003AF583E49322BB010FF8E58229F582E5F4
:104FC300833AF583E028F0225009C58229F8E58267
:104FD30026F622BBFE09C58229F8E22582F222F8D1
:104FE300EA2583F583E9932822BB010689828A8314
:104FF300F0225002F722BBFE01F322F8BB010DE5BC
:105003008229F582E5833AF583E8F0225006E92503
:1050130082C8F622BBFE05E92582C8F222EF8DF095
:10502300A4A8F0CF8CF0A428CE8DF0A42EFE22BC31
:10503300000BBE0029EF8DF084FFADF022E4CCF825
:1050430075F008EF2FFFEE33FEEC33FCEE9DEC988A
:105053004005FCEE9DFE0FD5F0E9E4CEFD22EDF810
:10506300F5F0EE8420D21CFEADF075F008EF2FFFB3
:10507300ED33FD4007985006D5F0F222C398FD0F9B
:10508300D5F0EA22C2D5EC30E709B2D5E4C39DFDE1
:10509300E49CFCEE30E715B2D5E4C39FFFE49EFE2B
:1050A300125032C3E49DFDE49CFC80031250323065
:1050B300D507C3E49FFFE49EFE22C5F0F8A3E028D2
:1050C300F0C5F0F8E582158270021583E038F0220E
:1050D300A3F8E0C5F025F0F0E58215827002158390
:1050E300E0C838F0E822BB010A89828A83E0F5F040
:1050F300A3E022500687F009E71922BBFE07E3F578
:10510300F009E3192289828A83E493F5F074019309
:1051130022E88FF0A4CC8BF0A42CFCE98EF0A42C15
:10512300FC8AF0EDA42CFCEA8EF0A4CDA8F08BF061
:10513300A42DCC3825F0FDE98FF0A42CCD35F0FC5F
:10514300EB8EF0A4FEA9F0EB8FF0A4CFC5F02ECD2B
:1051530039FEE43CFCEAA42DCE35F0FDE43CFC2210
:1051630075F008758200EF2FFFEE33FECD33CDCC03
:1051730033CCC58233C5829BED9AEC99E582984086
:105183000CF582EE9BFEED9AFDEC99FC0FD5F0D663
:10519300E4CEFBE4CDFAE4CCF9A88222B800C1B98D
:1051A3000059BA002DEC8BF084CFCECDFCE5F0CBCB
:1051B300F97818EF2FFFEE33FEED33FDEC33FCEB04
:1051C30033FB10D703994004EB99FB0FD8E5E4F9BF
:1051D300FA227818EF2FFFEE33FEED33FDEC33FCAC
:1051E300C933C910D7059BE99A4007EC9BFCE99AA0
:1051F300F90FD8E0E4C9FAE4CCFB2275F010EF2FE5
:10520300FFEE33FEED33FDCC33CCC833C810D707E4
:105213009BEC9AE899400AED9BFDEC9AFCE899F81F
:105223000FD5F0DAE4CDFBE4CCFAE4C8F922CFF4ED
:10523300CFCEF4CECDF4CDCCF4CC22EB9FF5F0EA77
:105243009E42F0E99D42F0EC6480C864809845F08A
:1052530022EB9FF5F0EA9E42F0E99D42F0E89C457F
:10526300F022E8600FECC313FCED13FDEE13FEEF29
:1052730013FFD8F122E8600FEFC333FFEE33FEEDE7
:1052830033FDEC33FCD8F122BB010789828A830208
:1052930054A15005E9F8025495BBFE05E9F8025400
:1052A300AD89828A830254B9BB010DE58229F58257
:1052B300E5833AF5830254A15007E92582F80254A5
:1052C30095BBFE07E92582F80254ADE58229F582F4
:1052D300E5833AF5830254B9BB010789828A8302C5
:1052E30053395005E9F80254FFBBFE05E9F80255AE
:1052F3000B22BB010DE58229F582E5833AF5830292
:1053030053395007E92582F80254FFBBFE07E9250C
:1053130082F802550B22BB010789828A830254D685
:105323005005E9F80254C9BBFE05E9F80254E289C5
:10533300828A830254EFECF0A3EDF0A3EEF0A3EF27
:10534300F022A8828583F0D083D08212535C12535B
:105353005C12535C12535CE473E493A3C583C5F0FE
:10536300C583C8C582C8F0A3C583C5F0C583C8C5B6
:1053730082C822BB010789828A830253455005E90B
:10538300F8025517BBFE05E9F802553022BB010DA3
:10539300E58229F582E5833AF5830253455007E90F
:1053A3002582F8025517BBFE07E92582F80255301E
:1053B30022A42582F582E5F03583F58322BB01071C
:1053C30089828A8302555B5005E9F8025549BBFE81
:1053D30005E9F802556D89828A8302557FBB010D69
:1053E300E58229F582E5833AF58302555B5007E9A7
:1053F3002582F8025549BBFE07E92582F802556D5F
:10540300E58229F582E5833AF58302557FBB0120C6
:10541300E58229F582E5833AF583D0F0D0E0F8D030
:10542300E0F9D0E0FAD0E0FBE8C0E0C0F002556458
:105433005018E92582F8D083D082D0E0F9D0E0FA81
:10544300D0E0FBC082C083025552BBFE18E925821F
:10545300F8D083D082D0E0F9D0E0FAD0E0FBC0826C
:10546300C08302557622D083D082F8E493701274FD
:105473000193700DA3A393F8740193F5828883E4D9
:10548300737402936860EFA3A3A380DF8A83898286
:10549300E473E6FC08E6FD08E6FE08E6FF22E0FC0E
:1054A300A3E0FDA3E0FEA3E0FF22E2FC08E2FD0887
:1054B300E2FE08E2FF22E493FC740193FD7402937D
:1054C300FE740393FF22E6FB08E6F908E6FA08E612
:1054D300CBF822E0F8A3E0F9A3E0FAA3E0FB22E291
:1054E300FB08E2F908E2FA08E2CBF822E493F87445
:1054F3000193F9740293FA740393FB22ECF608ED1B
:10550300F608EEF608EFF622ECF208EDF208EEF2FA
:1055130008EFF222D083D082E493F608740193F665
:1055230008740293F608740393F6740473D083D05B
:1055330082E493F208740193F208740293F20874FC
:105543000393F2740473E6FB08E6FA08E6F922EB28
:10555300F608EAF608E9F622E0FBA3E0FAA3E0F98D
:1055630022EBF0A3EAF0A3E9F022E2FB08E2FA0857
:10557300E2F922EBF208EAF208E9F222E493FB747F
:105583000193FA740293F922900A79EBF0A3EAF0FB
:10559300A3E9F0900A79E0FBA3E0FAA3E0F97582AE
:1055A30006758300124F8CFFEFC39440402A900A84
:1055B30079E0FBA3E0FAA3E0F9758206758300E4C2
:1055C300124FFE900A79E0FBA3E0FAA3E0F975829B
:1055D3008B758300E4124FFE900A79E0FBA3E0FA97
:1055E300A3E0F9758204758300124F8CFF900A794A
:1055F300E0FBA3E0FAA3E0F9758205758300EF12DF
:105603004FFE900A79E0FBA3E0FAA3E0F975820369
:10561300758300124F8CFF900A79E0FBA3E0FAA395
:10562300E0F9758204758300EF124FFE900A79E06A
:10563300FBA3E0FAA3E0F9758202758300124F8C95
:10564300FF900A79E0FBA3E0FAA3E0F97582037502
:105653008300EF124FFE900A79E0FBA3E0FAA3E088
:10566300F9124F73FF900A79E0FBA3E0FAA3E0F984
:10567300758202758300EF124FFE900A79E0FBA357
:10568300E0FAA3E0F9124F73FF900A79E0FBA3E07D
:10569300FAA3E0F97582067583007401124FB9FE0F
:1056A300EEFD7C00900A79E0FBA3E0FAA3E0F9E9C0
:1056B3002409F9EA3400FAE92DF9EA3CFAEF124F2A
:1056C300EC900A79E0FBA3E0FAA3E0F975828B750D
:1056D3008300124F8CFFEF60030259EF900A79E0C9
:1056E300FBA3E0FAA3E0F9758202758300124F8CE5
:1056F300FFEFB44B35900A79E0FBA3E0FAA3E0F99E
:10570300758203758300124F8CFFEFB44F1C90001A
:10571300247401F0900A79E0FBA3E0FAA3E0F975A1
:10572300828B7583007401124FFE900A79E0FBA30C
:10573300E0FAA3E0F9758202758300124F8CFFEF44
:1057430064437050900A79E0FBA3E0FAA3E0F97593
:105753008203758300124F8CFFEFB45437900A799C
:10576300E0FBA3E0FAA3E0F9758204758300124F0E
:105773008CFFEFB42B1E900027E4F0900A79E0FB36
:10578300A3E0FAA3E0F975828B7583007401124FCD
:10579300FE025A4F900A79E0FBA3E0FAA3E0F97501
:1057A3008202758300124F8CFFEF644D7050900A94
:1057B30079E0FBA3E0FAA3E0F97582037583001295
:1057C3004F8CFFEFB44337900A79E0FBA3E0FAA3D1
:1057D300E0F9758204758300124F8CFFEFB42B1E22
:1057E300900027E4F0900A79E0FBA3E0FAA3E0F944
:1057F30075828B7583007401124FFE025A4F900A13
:1058030079E0FBA3E0FAA3E0F97582027583001245
:105813004F8CFFEF644360030258DF900A79E0FB8B
:10582300A3E0FAA3E0F9758203758300124F8CFF9E
:10583300EF644360030258DF900A79E0FBA3E0FAC8
:10584300A3E0F9758204758300124F8CFFEF642B7C
:1058530060030258DF900A79E0FBA3E0FAA3E0F9C2
:1058630075828B7583007402124FFE900A79E0FBF8
:10587300A3E0FAA3E0F975824A7583007402124F1C
:10588300FE900A79E0FBA3E0FAA3E0F975824B7579
:105893008300742B124FFE900A79E0FBA3E0FAA376
:1058A300E0F975824C7583007443124FFE900A79B8
:1058B300E0FBA3E0FAA3E0F975824D75830074431E
:1058C300124FFE900A79E0FBA3E0FAA3E0F9758298
:1058D300067583007403124FFE025A4F900A79E053
:1058E300FBA3E0FAA3E0F9758202758300124F8CE3
:1058F300FFEF64506003025A4F900A79E0FBA3E084
:10590300FAA3E0F9758203758300124F8CFFEF64ED
:10591300496003025A4F900A79E0FBA3E0FAA3E03F
:10592300F9758204758300124F8CFFEF64436003A3
:10593300025A4F900A79E0FBA3E0FAA3E0F97582DB
:1059430005758300124F8CFFEF642B6003025A4FDF
:10595300900A79E0FBA3E0FAA3E0F975828B7583E3
:10596300007403124FFE900A79E0FBA3E0FAA3E070
:10597300F975824A7583007403124FFE900A79E029
:10598300FBA3E0FAA3E0F975824B758300742B1235
:105993004FFE900A79E0FBA3E0FAA3E0F975824C8D
:1059A3007583007443124FFE900A79E0FBA3E0FA7B
:1059B300A3E0F975824D7583007449124FFE900A76
:1059C30079E0FBA3E0FAA3E0F975824E75830074D6
:1059D30050124FFE900A79E0FBA3E0FAA3E0F975B9
:1059E30082067583007404124FFE8060900A79E08A
:1059F300FBA3E0FAA3E0F975828B758300124F8C49
:105A0300FFEFD394014045900A79E0FBA3E0FAA3AA
:105A1300E0F9124F73FF900A79E0FBA3E0FAA3E0E9
:105A2300F9758206758300124F8CFEEEFD7C0090A3
:105A33000A79E0FBA3E0FAA3E0F9E9244AF9EA349E
:105A430000FAE92DF9EA3CFAEF124FEC900A79E0FB
:105A5300FBA3E0FAA3E0F9758202758300124F8C71
:105A6300FFEF640A6003025B47900A79E0FBA3E05F
:105A7300FAA3E0F9758203758300124F8CFFEF647C
:105A83000D6003025B47900A79E0FBA3E0FAA3E011
:105A9300F9758206758300124F8CFFEFD394024091
:105AA30079900A79E0FBA3E0FAA3E0F975828B759C
:105AB3008300124F8CFFEFD39401405E900A79E08C
:105AC300FBA3E0FAA3E0F9758207758300124F8CFC
:105AD300FFEF64016044900A79E0FBA3E0FAA3E0DE
:105AE300F9758206758300124F8CFFEF24FEFF9039
:105AF3000A79E0FBA3E0FAA3E0F975820975830054
:105B0300EF124FFE900A79E0FBA3E0FAA3E0F975E8
:105B130082077583007401124FFE900A79E0FBA39C
:105B2300E0FAA3E0F9758206758300E4124FFE9054
:105B33000A79E0FBA3E0FAA3E0F975828B75830091
:105B4300E4124FFE2290013EEBF0A3EAF0A3E9F04A
:105B5300900270E4F0900271E4F07B007A00790027
:105B6300900272EBF0A3EAF0A3E9F07B017A0179EA
:105B730041900275EBF0A3EAF0A3E9F090013EE057
:105B8300FBA3E0FAA3E0F9900272EBF0A3EAF0A31F
:105B9300E9F0900272E0FBA3E0FAA3E0F9124F737D
:105BA300FFEF7003025F90900272E0FBA3E0FAA3A1
:105BB300E0F9124F73FFEF645C6003025C679002CD
:105BC30072E0FBA3E475F0011250BDA9F0FA124F85
:105BD30073FFEF1254695C0B6E5BE6725C31740009
:105BE300005C57900270E0FF04F0EF3395E0FE7421
:105BF300942FF58274033EF583740DF0900273E4E1
:105C030075F0011250BD808A900270E0FF04F0EF3E
:105C13003395E0FE74942FF58274033EF583740A82
:105C2300F0900273E475F0011250BD025B9590028F
:105C330070E0FF04F0EF3395E0FE74942FF5827467
:105C4300033EF5837409F0900273E475F00112507A
:105C5300BD025B95900273E475F0011250BD025BC7
:105C630095025B95900272E0FBA3E0FAA3E0F912C0
:105C73004F73FFEF64256003025F60900272E0FBE5
:105C8300A3E475F0011250BDA9F0FA124F73FFEFB0
:105C93001254695CB2435E3C535D99585CB2635CD9
:105CA300F6645EAD665E3C735D997800005F50906C
:105CB3000275E0FBA3E475F0011250D3A9F0FA12C8
:105CC3004F73FF900271EFF0900271E0FF9002704A
:105CD300E0FE04F0EEFD3395E0FC74942DF5827440
:105CE300033CF583EFF0900273E475F0011250BDAD
:105CF300025B95900275E0FBA3E475F0021250D3AA
:105D0300A9F0FA1250E9FFAEF0EE3395E0FDFC90F6
:105D1300016C12533990016CE0FCA3E0FDA3E0FE9B
:105D2300A3E0FF7B017A017970900860740AF01296
:105D33005FAF7B017A017970900169EBF0A3EAF020
:105D4300A3E9F0900169E0FBA3E0FAA3E0F9124FA5
:105D530073FFEF6034900169E0FBA3E0FAA3E0F97D
:105D6300124F73FF900270E0FE04F0EEFD3395E0F6
:105D7300FC74942DF58274033CF583EFF090016A73
:105D8300E475F0011250BD80BA900273E475F0011E
:105D93001250BD025B95900275E0FBA3E475F0021F
:105DA3001250D3A9F0FA1250E9FFAEF0EE3395E0AA
:105DB300FDFC90016C12533990016CE0FCA3E0FDF3
:105DC300A3E0FEA3E0FF7B017A0179709008607481
:105DD30010F0125FAF7B017A017970900169EBF0EB
:105DE300A3EAF0A3E9F0900169E0FBA3E0FAA3E0E2
:105DF300F9124F73FFEF6034900169E0FBA3E0FAFF
:105E0300A3E0F9124F73FF900270E0FE04F0EEFD81
:105E13003395E0FC74942DF58274033CF583EFF025
:105E230090016AE475F0011250BD80BA900273E4E8
:105E330075F0011250BD025B95900275E0FBA3E47F
:105E430075F0031250D3A9F0FA1253C0900169EB15
:105E5300F0A3EAF0A3E9F0900169E0FBA3E0FAA361
:105E6300E0F9124F73FFEF6034900169E0FBA3E0A8
:105E7300FAA3E0F9124F73FF900270E0FE04F0EE14
:105E8300FD3395E0FC74942DF58274033CF583EFA8
:105E9300F090016AE475F0011250BD80BA9002736C
:105EA300E475F0011250BD025B95900275E0FBA30F
:105EB300E475F0021250D3A9F0FA1250E9FFAEF0E4
:105EC300EE3395E0FDFC90016C12533990016CE0C8
:105ED300FCA3E0FDA3E0FEA3E0FF7B017A01797060
:105EE300900860740AF0125FAF7B017A01797090B9
:105EF3000169EBF0A3EAF0A3E9F0900169E0FBA3E9
:105F0300E0FAA3E0F9124F73FFEF6034900169E008
:105F1300FBA3E0FAA3E0F9124F73FF900270E0FED7
:105F230004F0EEFD3395E0FC74942DF58274033C8C
:105F3300F583EFF090016AE475F0011250BD80BA69
:105F4300900273E475F0011250BD025B95900273E9
:105F5300E475F0011250BD025B95025B95900272ED
:105F6300E0FBA3E475F0011250D3A9F0FA124F73CA
:105F7300FF900270E0FE04F0EEFD3395E0FC7494B4
:105F83002DF58274033CF583EFF0025B959002706C
:105F9300E0FF900393EFF07B017A03799490038FF2
:105FA300EBF0A3EAF0A3E9F0127AC12290085912A8
:105FB300533990085DEBF0A3EAF0A3E9F090086988
:105FC300E4F090086AE4F0A3E4F090085DE0FBA33A
:105FD300E0FAA3E0F990086CEBF0A3EAF0A3E9F090
:105FE300900859E0FCA3E0FDA3E0FEA3E0FFEC4D25
:105FF3004E4F703090086CE0FBA3E475F001125033
:10600300D3A9F0FA7430124FEC90086CE0FBA3E0D4
:10601300FAA3E0F9E4124FEC90085DE0FBA3E0FA89
:10602300A3E0F922900859E0FCA3E0FDA3E0FEA35E
:10603300E0FF90086AEEF0A3EFF0900860E0FFEF56
:1060430012546961D50A60533260C3340000638A15
:1060530090086AE0FEA3E0FFEEC4F854F0C868FEBF
:10606300EFC4540F48FFEF540FFF128CB390086C2A
:10607300E0FBA3E475F0011250D3A9F0FAEF124F3D
:10608300EC90086AE0FEA3E0FFEF540FFF128CB31D
:1060930090086CE0FBA3E475F0011250D3A9F0FA69
:1060A300EF124FEC90086CE0FBA3E0FAA3E0F9E4F5
:1060B300124FEC90085DE0FBA3E0FAA3E0F9222283
:1060C30090086AE0FEA3E0FFEEC4540FFF7E00EFEA
:1060D300540FFF128CB390086CE0FBA3E475F0013E
:1060E3001250D3A9F0FAEF124FEC90086AE0FEA326
:1060F300E0FFEEFF7E00EF540FFF128CB390086CAD
:10610300E0FBA3E475F0011250D3A9F0FAEF124FAC
:10611300EC90086AE0FEA3E0FFEEC4540FFF7E009C
:10612300EF540FFF128CB390086CE0FBA3E475F0FF
:10613300011250D3A9F0FAEF124FEC90086AE0FE77
:10614300A3E0FFEEFF7E00EF540FFF128CB3900825
:106153006CE0FBA3E475F0011250D3A9F0FAEF123F
:106163004FEC90086AE0FEA3E0FFEEC4F854F0C8D9
:1061730068FEEFC4540F48FFEF540FFF128CB39027
:10618300086CE0FBA3E475F0011250D3A9F0FAEF19
:10619300124FEC90086AE0FEA3E0FFEF540FFF12EA
:1061A3008CB390086CE0FBA3E475F0011250D3A903
:1061B300F0FAEF124FEC90086CE0FBA3E0FAA3E0D7
:1061C300F9E4124FEC90085DE0FBA3E0FAA3E0F9D9
:1061D30022227F007E007D007C00900859E0F8A316
:1061E300E0F9A3E0FAA3E0FBC312523E5034900857
:1061F3006CE0FBA3E475F0011250D3A9F0FA742DFF
:10620300124FEC900859E0FCA3E0FDA3E0FEA3E0ED
:10621300FF7BFF7AFF79FF78FF1251149008591220
:106223005339900861125345000186A0900861E03C
:10623300FCA3E0FDA3E0FEA3E0FF900859E0F8A370
:10624300E0F9A3E0FAA3E0FBD312523E4014900816
:1062530061E0FCA3E0FDA3E0FEA3E0FF9008591278
:1062630053397F007E007D007C00900861E0F8A335
:10627300E0F9A3E0FAA3E0FBD312523E500302631A
:106283006E900861E0F8A3E0F9A3E0FAA3E0FB90C5
:106293000859E0FCA3E0FDA3E0FEA3E0FF120046E3
:1062A300900865125339900865E0FCA3E0FDA3E074
:1062B300FEA3E0FFEC4D4E4F700B900869E0FFEF3B
:1062C300700302634C900865E0FCA3E0FDA3E0FECD
:1062D300A3E0FFEF2430FF90086CE0FBA3E475F02C
:1062E300011250D3A9F0FAEF124FEC900859E0FCD9
:1062F300A3E0FDA3E0FEA3E0FFC004C005C006C009
:1063030007900861E0FCA3E0FDA3E0FEA3E0FF909B
:106313000865E0F8A3E0F9A3E0FAA3E0FB12511447
:10632300A804A905AA06AB07D007D006D005D00458
:10633300C3EF9BFFEE9AFEED99FDEC98FC90085994
:106343001253399008697401F0900861E0FCA3E0EE
:10635300FDA3E0FEA3E0FF7B0A7A00790078001238
:10636300004690086112533902626590086CE0FBA5
:10637300A3E0FAA3E0F9E4124FEC90085DE0FBA37D
:10638300E0FAA3E0F9222290086CE0FBA3E475F0A5
:10639300011250D3A9F0FA7430124FEC90086CE05C
:1063A300FBA3E0FAA3E0F9E4124FEC90085DE0FBF5
:1063B300A3E0FAA3E0F92290086FEBF0A3EAF0A3BD
:1063C300E9F09008791253450000000090087D120F
:1063D300534500000000900881125345000000005F
:1063E30090086FE0FBA3E0FAA3E0F912528B780365
:1063F300125265EF543FFFEE5400FEED5400FDECE6
:106403005400FC90087D12533990087DE0F8A3E016
:10641300F9A3E0FAA3E0FBC374409BFFE49AFEE414
:1064230099FDE498FC90088112533990086FE0FBC2
:10643300A3E0FAA3E0F9C003C002C00112528BC06B
:1064430004C005C006C007900875E0FCA3E0FDA3E7
:10645300E0FEA3E0FF7803125278A804A905AA0678
:10646300AB07D007D006D005D004EF2BFFEE3AFEE2
:10647300ED39FDEC38FCD001D002D0031252DB9091
:106483000875E0FCA3E0FDA3E0FEA3E0FF780312A0
:10649300527890086FE0FBA3E0FAA3E0F9125319D6
:1064A300C3125254503C90086FE0FBA3E0FAA3E000
:1064B300F97582047583001252AB7B017A0079006F
:1064C3007800EF2BFFEE3AFEED39FDEC38FC900837
:1064D3006FE0FBA3E0FAA3E0F97582047583001271
:1064E30052F590086FE0FBA3E0FAA3E0F9E9240476
:1064F300F9EA3400FAC003C002C00112528BC0048F
:10650300C005C006C007900875E0FCA3E0FDA3E04A
:10651300FEA3E0FF781D125265A804A905AA06ABE5
:1065230007D007D006D005D004EF2BFFEE3AFEEDDF
:1065330039FDEC38FCD001D002D0031252DB9008B5
:1065430081E0FCA3E0FDA3E0FEA3E0FF900875E07B
:10655300F8A3E0F9A3E0FAA3E0FBC31252545003FB
:106563000266D390086FE0FBA3E0FAA3E0F9E92405
:1065730018F9EA3400FA90087DE0FCA3E0FDA3E0FB
:10658300FEA3E0FFE92FF9EA3EFAEB3DFBC003C0AF
:1065930002C001900872E0FBA3E0FAA3E0F99009BE
:1065A30096EBF0A3EAF0A3E9F0900881E0FCA3E006
:1065B300FDA3E0FEA3E0FF900999EEF0A3EFF0D076
:1065C30001D002D003128B8A90086FE0FBA3E0FA9C
:1065D300A3E0F9E92408F9EA3400FAC003C002C0D1
:1065E3000190086FE0FBA3E0FAA3E0F9E92418F9AE
:1065F300EA3400FA90027BEBF0A3EAF0A3E9F0D0CF
:1066030001D002D003120096900881E0FCA3E0FDC4
:10661300A3E0FEA3E0FF900879125339900879E0D4
:10662300FCA3E0FDA3E0FEA3E0FFEF2440FFEE3474
:1066330000FEED3400FDEC3400FC900875E0F8A397
:10664300E0F9A3E0FAA3E0FBC312525440769008AA
:106653006FE0FBA3E0FAA3E0F9E92408F9EA3400C8
:10666300FAC003C002C001900879E0FCA3E0FDA3D7
:10667300E0FEA3E0FF900872E0FBA3E0FAA3E0F9D9
:10668300E92FF9EA3EFAEB3DFB90027BEBF0A3EA3C
:10669300F0A3E9F0D001D002D0031200969008795C
:1066A300E0FCA3E0FDA3E0FEA3E0FFEF2440FFEE48
:1066B3003400FEED3400FDEC3400FC9008791253F5
:1066C3003902661F90087D12534500000000800ABE
:1066D3009008791253450000000090086FE0FBA377
:1066E300E0FAA3E0F9E92418F9EA3400FA90087D06
:1066F300E0FCA3E0FDA3E0FEA3E0FFE92FF9EA3EFF
:10670300FAEB3DFBC003C002C001900879E0FCA393
:10671300E0FDA3E0FEA3E0FF900872E0FBA3E0FA34
:10672300A3E0F9E92FF9EA3EFAEB3DFB900996EB7A
:10673300F0A3EAF0A3E9F0900879E0FCA3E0FDA35D
:10674300E0FEA3E0FFAB07AA06900875E0FCA3E018
:10675300FDA3E0FEA3E0FFC3EF9BFFEE9AFE9009CB
:1067630099EEF0A3EFF0D001D002D003128B8A226E
:10677300900A73EBF0A3EAF0A3E9F0900A73E0FB4D
:10678300A3E0FAA3E0F9124F73FF900A73E0FBA3AF
:10679300E0FAA3E0F9758201758300EF124FFE90D2
:1067A3000A73E0FBA3E0FAA3E0F9758202758300A4
:1067B300124F8CFF900A73E0FBA3E0FAA3E0F9EF1A
:1067C300124FEC900A73E0FBA3E0FAA3E0F97582A1
:1067D30006758300124F8CFFEF600302690D900A68
:1067E30073E0FBA3E0FAA3E0F9758204758300125A
:1067F3004F8CFF900A73E0FBA3E0FAA3E0F97582E4
:1068030001758300124F8CFEEE6F6003026A729073
:106813000A73E0FBA3E0FAA3E0F975820575830030
:10682300124F8CFF900A73E0FBA3E0FAA3E0F91286
:106833004F73FEEE6F6003026A72900A73E0FBA36C
:10684300E0FAA3E0F97582067583007401124FFE26
:10685300900A73E0FBA3E0FAA3E0F9758203758362
:1068630000740F124FFE900A73E0FBA3E0FAA3E05B
:10687300F9E9240CF9EA3400FAC003C002C001901C
:106883000A73E0FBA3E0FAA3E0F9758209758300BC
:10689300125410900A73E0FBA3E0FAA3E0F97582A7
:1068A30004758300124F8CFF900A73E0FBA3E0FA98
:1068B300A3E0F97582097583001253E0EF124FECE0
:1068C300900A73E0FBA3E0FAA3E0F97582057583F0
:1068D30000124F8CFF900A73E0FBA3E0FAA3E0F9E8
:1068E3007582097583001253E0758201758300EF89
:1068F300124FFE900A73E0FBA3E0FAA3E0F975825E
:10690300087583007401124FFE22900A73E0FBA303
:10691300E0FAA3E0F97582087583007401124FB998
:10692300900A73E0FBA3E0FAA3E0F9124F73FF9020
:106933000A73E0FBA3E0FAA3E0F97582097583000B
:106943001253E0C003C002C001900A73E0FBA3E04E
:10695300FAA3E0F9758208758300124F8CFED0010B
:10696300D002D0038E82758300EF124FFE900A731C
:10697300E0FBA3E0FAA3E0F9758208758300124FE8
:106983008CFFEF6402705F900A73E0FBA3E0FAA34D
:10699300E0F9758202758300124F8CFFEF2402FF2A
:1069A300900A73E0FBA3E0FAA3E0F9758203758311
:1069B30000EF124FFE900A73E0FBA3E0FAA3E0F9A5
:1069C300758203758300124F8CFFEFC3941040163A
:1069D300900A73E0FBA3E0FAA3E0F97582037583E1
:1069E30000740F124FFE900A73E0FBA3E0FAA3E0DA
:1069F300F9758203758300124F8CFF900A73E0FBD5
:106A0300A3E0FAA3E0F9758208758300124F8CFEA8
:106A1300EEC39F405A900A73E0FBA3E0FAA3E0F9A8
:106A2300758207758300124F8CFFEF640160169027
:106A33000A73E0FBA3E0FAA3E0F97582077583000C
:106A43007401124FFE900A73E0FBA3E0FAA3E0F98E
:106A5300758208758300E4124FFE900A73E0FBA36E
:106A6300E0FAA3E0F9758206758300E4124FFE2273
:106A73009008B0EBF0A3EAF0A3E9F09008BA125340
:106A830045000000009008BE12534500000000902E
:106A930008B6E0FCA3E0FDA3E0FEA3E0FF9008BE80
:106AA300E0F8A3E0F9A3E0FAA3E0FBC312525440D9
:106AB30003026CAD7F047E007D007C009008BAE089
:106AC300F8A3E0F9A3E0FAA3E0FB1251149008B392
:106AD300E0FBA3E0FAA3E0F98F828E831252ABEFBF
:106AE30054FFFFEE5400FEED5400FDEC5400FCC0D7
:106AF300079008BEE0FCA3E0FDA3E0FEA3E0FF9047
:106B030008B0E0FBA3E0FAA3E0F98F828E83D007FD
:106B1300EF124FFE7F047E007D007C009008BAE0F8
:106B2300F8A3E0F9A3E0FAA3E0FB1251149008B331
:106B3300E0FBA3E0FAA3E0F98F828E831252AB78D5
:106B430008125265EF54FFFFEE5400FEED5400FDB2
:106B5300EC5400FCC0079008BEE0FCA3E0FDA3E0FA
:106B6300FEA3E0FFEF2401FFEE3400FE9008B0E047
:106B7300FBA3E0FAA3E0F98F828E83D007EF124FD5
:106B8300FE7F047E007D007C009008BAE0F8A3E05D
:106B9300F9A3E0FAA3E0FB1251149008B3E0FBA3BE
:106BA300E0FAA3E0F98F828E831252AB781012526F
:106BB30065EF54FFFFEE5400FEED5400FDEC54006E
:106BC300FCC0079008BEE0FCA3E0FDA3E0FEA3E049
:106BD300FFEF2402FFEE3400FE9008B0E0FBA3E0D9
:106BE300FAA3E0F98F828E83D007EF124FFE7F0462
:106BF3007E007D007C009008BAE0F8A3E0F9A3E0F2
:106C0300FAA3E0FB1251149008B3E0FBA3E0FAA34C
:106C1300E0F98F828E831252AB7818125265EF54CB
:106C2300FFFFEE5400FEED5400FDEC5400FCC007E2
:106C33009008BEE0FCA3E0FDA3E0FEA3E0FFEF2489
:106C430003FFEE3400FE9008B0E0FBA3E0FAA3E0FC
:106C5300F98F828E83D007EF124FFE9008BAE0FCC3
:106C6300A3E0FDA3E0FEA3E0FF7B017A00790078B7
:106C730000EF2BFFEE3AFEED39FDEC38FC9008BA3D
:106C83001253399008BEE0FCA3E0FDA3E0FEA3E0AD
:106C9300FFEF2404FFEE3400FEED3400FDEC34007E
:106CA300FC9008BE125339026A92229008C2EBF09C
:106CB300A3EAF0A3E9F09008CC12534500000000CA
:106CC3009008D0125345000000009008C8E0FCA3D0
:106CD300E0FDA3E0FEA3E0FF9008D0E0F8A3E0F915
:106CE300A3E0FAA3E0FBC31252544003026E9D904B
:106CF30008D0E0FCA3E0FDA3E0FEA3E0FFEF240146
:106D0300FFEE3400FE9008C5E0FBA3E0FAA3E0F930
:106D13008F828E83124F8CFFE4FCFDFE78081252A3
:106D230078C004C005C006C0079008D0E0FCA3E00B
:106D3300FDA3E0FEA3E0FF9008C5E0FBA3E0FAA3F8
:106D4300E0F98F828E83124F8CFFAB07E4FAF9F8D8
:106D5300D007D006D005D004EF4BFFEE4AFEED4935
:106D6300FDEC48FCC004C005C006C0079008D0E095
:106D7300FCA3E0FDA3E0FEA3E0FFEF2402FFEE345B
:106D830000FE9008C5E0FBA3E0FAA3E0F98F828E32
:106D930083124F8CFFE4FCFDFE7810125278A80496
:106DA300A905AA06AB07D007D006D005D004EB4F40
:106DB300FFEA4EFEE94DFDE84CFCC004C005C006E9
:106DC300C0079008D0E0FCA3E0FDA3E0FEA3E0FF32
:106DD300EF2403FFEE3400FE9008C5E0FBA3E0FAC6
:106DE300A3E0F98F828E83124F8CFFE4FCFDFE78C3
:106DF30018125278A804A905AA06AB07D007D00633
:106E0300D005D004EB4FFFEA4EFEE94DFDE84CFC04
:106E1300C004C005C006C0077F047E007D007C005F
:106E23009008CCE0F8A3E0F9A3E0FAA3E0FB125149
:106E3300149008C2E0FBA3E0FAA3E0F98F828E83EB
:106E4300D007D006D005D0041252F59008CCE0FC50
:106E5300A3E0FDA3E0FEA3E0FF7B017A00790078C5
:106E630000EF2BFFEE3AFEED39FDEC38FC9008CC39
:106E73001253399008D0E0FCA3E0FDA3E0FEA3E0A9
:106E8300FFEF2404FFEE3400FEED3400FDEC34008C
:106E9300FC9008D0125339026CCD22900929EBF0F3
:106EA300A3EAF0A3E9F0900929E0FBA3E0FAA3E049
:106EB300F9124F73FF90092FEFF0900930E4F0902F
:106EC3000929E0FBA3E0FAA3E0F9758201758300C9
:106ED300124F8CFF900931EFF0900932E4F09009E2
:106EE3002CE4F090092CE0FFEFC3940640030270FA
:106EF3004D90092CE0FF900931E0FEEEA8070880D1
:106F030002C313D8FCFFEF5401FF90092DEFF0905B
:106F1300092CE0FF90092FE0FEEEA807088002C3CA
:106F230013D8FCFFEF5401FF90092EEFF090092DC9
:106F3300E0FFEF6401600302704490092CE0FFEF6F
:106F43001254696F5C006F7F016FA6026FCE036FEF
:106F5300F704701E0500007044900932E0FFEF440F
:106F630001FF900932EFF0900930E0FF90092EE025
:106F7300FEEF4EFF900930EFF0027044900932E0CB
:106F8300FFEF4402FF900932EFF0900930E0FF90E9
:106F9300092EE0FEEE25E0FEEF4EFF900930EFF004
:106FA300027044900932E0FFEF4404FF900932EF8E
:106FB300F0900930E0FF90092EE0FEEE25E025E099
:106FC300FEEF4EFF900930EFF08076900932E0FF3C
:106FD300EF4408FF900932EFF0900930E0FF900989
:106FE3002EE0FEEE33333354F8FEEF4EFF900930BC
:106FF300EFF0804D900932E0FFEF4410FF9009322B
:10700300EFF0900930E0FF90092EE0FEEEC454F05B
:10701300FEEF4EFF900930EFF08026900932E0FF3B
:10702300EF4420FF900932EFF0900930E0FF900920
:107033002EE0FEEEC43354E0FEEF4EFF900930EF36
:10704300F090092CE004F0026EE6900930E0FF9026
:107053000929E0FBA3E0FAA3E0F9EF124FEC900952
:1070630032E0FF900929E0FBA3E0FAA3E0F975827F
:1070730001758300EF124FFE229007DFEBF0A3EAC6
:10708300F0A3E9F09007E2EDF07BFF7A8A79E3C0A1
:1070930003C002C0017B017A0779E4A801AC02AD09
:1070A30003D001D002D0037E007F10124F4D900712
:1070B300DFE0FBA3E0FAA3E0F99007F4EBF0A3EA27
:1070C300F0A3E9F09007F4E0FBA3E0FAA3E0F9757D
:1070D3008204758300124F8CFF9007F7EFF090073F
:1070E300F7E0FFEF12546971060071910171970285
:1070F300719D0371A395720696721D9871BA9900DA
:107103000072389007F4E0FBA3E0FAA3E0F975827C
:1071130003758300124F8CFF128DA69007F4E0FBDA
:10712300A3E0FAA3E0F9758204758300124F8CFF84
:10713300128DA69007E3E4F09007F4E0FBA3E0FAD6
:10714300A3E0F9758202758300124F8CFFEF24FED2
:10715300FF9007E3E0FEEEC39F40030272389007FF
:10716300F4E0FBA3E0FAA3E0F9E92405F9EA34002B
:10717300FA9007E3E0FF7E00E92FF9EA3EFA124FA7
:1071830073FF128DA69007E3E004F080AB227F47E4
:10719300128DA6227F44128DA6227F52128DA62223
:1071A3009007F4E0FBA3E0FAA3E0F9E92405F9EA88
:1071B3003400FA128BD2229007F4E0FBA3E0FAA387
:1071C300E0F9758206758300124F8CFFEF540FFFB1
:1071D3009009D8EFF07BFF7A8A79A3C003C002C07D
:1071E300017BFF7A8A79B1900141EBF0A3EAF0A326
:1071F300E9F0D001D002D003125B487FBC7E0212BB
:10720300880F229007F4E0FBA3E0FAA3E0F9E92456
:1072130005F9EA3400FA127D45229007F4E0FBA356
:10722300E0FAA3E0F9E92405F9EA3400FA9007E269
:10723300E0FD128B42229008D4EBF0A3EAF0A3E91D
:10724300F09008DC1253450000FFFF9008E1E4F0E2
:10725300A3E4F09008E3E4F0A3E4F09008E1E4F0A1
:10726300A3E4F09008DAE0FEA3E0FF9008E1E0FC7D
:10727300A3E0FDC3ED9FEC9E40030273879008D704
:10728300E0FBA3E0FAA3E0F9124F73FFEF54FFFF13
:107293009008E0EFF09008D8E475F0011250BD902B
:1072A30008DCE0F8A3E0F9A3E0FAA3E0FB9008E030
:1072B300E0FFE4FCFDFEEB6FFFEA6EFEE96DFDE827
:1072C3006CFC9008DC1253399008E3E4F0A3E4F07B
:1072D3009008E3E0FEA3E0FFC3EF9408EE6480941C
:1072E3008040030273769008DCE0FCA3E0FDA3E09A
:1072F300FEA3E0FFEF5401FFEE5400FEED5400FD4A
:10730300EC5400FCEC4D4E4F603F9008DCE0FCA3D6
:10731300E0FDA3E0FEA3E0FF78011252659008DCD4
:107323001253399008DCE0FCA3E0FDA3E0FEA3E0E8
:10733300FFEF6401FFEE64A0FEED6400FDEC64006A
:10734300FC9008DC12533980199008DCE0FCA3E0C0
:10735300FDA3E0FEA3E0FF78011252659008DC1262
:1073630053399008E4E004F070069008E3E004F079
:107373000272D39008E2E004F070069008E1E004A2
:10738300F00272669008DCE0FCA3E0FDA3E0FEA33C
:10739300E0FF9008E0EFF09008DCE0FCA3E0FDA341
:1073A300E0FEA3E0FF9008D4E0FBA3E0FAA3E0F93A
:1073B300EF124FEC9008DCE0FCA3E0FDA3E0FEA39A
:1073C300E0FF78081252659008D4E0FBA3E0FAA32B
:1073D300E0F9758201758300EF124FFE2290088554
:1073E300EBF0A3EAF0A3E9F090088B1253450000F9
:1073F300000090088F12534500000000900885E0BC
:10740300FBA3E0FAA3E0F912528B7803125265EF63
:10741300543FFFEE5400FEED5400FDEC5400FC908D
:10742300088B1253397F387E007D007C0090088BD7
:10743300E0F8A3E0F9A3E0FAA3E0FBC3125254502F
:107443001E90088BE0F8A3E0F9A3E0FAA3E0FBC3E6
:1074530074389BFFE49AFEE499FDE498FC801C9049
:10746300088BE0F8A3E0F9A3E0FAA3E0FBC3747888
:107473009BFFE49AFEE499FDE498FC90088F125375
:10748300397B017A087993C003C002C00190088553
:10749300E0FBA3E0FAA3E0F99008B3EBF0A3EAF072
:1074A300A3E9F09008B612534500000008D001D0BC
:1074B30002D003126A73900885E0FBA3E0FAA3E00D
:1074C300F9C003C002C0017B017A077900900872FA
:1074D300EBF0A3EAF0A3E9F090088FE0FCA3E0FD52
:1074E300A3E0FEA3E0FF900875125339D001D00248
:1074F300D0031263BA900885E0FBA3E0FAA3E0F996
:10750300C003C002C0017B017A087993900872EB33
:10751300F0A3EAF0A3E9F0900875125345000000C8
:1075230008D001D002D0031263BA900888E0FBA30D
:10753300E0FAA3E0F9C003C002C001900885E0FBB4
:10754300A3E0FAA3E0F9E92408F9EA3400FA900881
:10755300B3EBF0A3EAF0A3E9F09008B612534500A9
:10756300000010D001D002D003126A732290098365
:10757300EBF0A3EAF0A3E9F0900986EDF09009831C
:10758300E0FBA3E0FAA3E0F9124F73FF900987EF42
:10759300F0900983E0FBA3E0FAA3E0F9758201759B
:1075A3008300124F8CFF900988EFF0900983E0FB72
:1075B300A3E0FAA3E0F9758202758300124F8CFFF2
:1075C300900989EFF0900988E0FFEF1313543FFF10
:1075D300EF540FFF90098AEFF0900986E4F09009C9
:1075E300D8E0FFEFB40308900987E0FF12899E906B
:1075F30009D8E0FFEFB403057F2D128DA69009D8BB
:10760300E0FFEFB40308900988E0FF12899E900918
:10761300D8E0FFEFB403057F2D128DA69009D8E0C3
:10762300FFEFB40308900989E0FF12899E9009D8FF
:10763300E0FFEFB403057F20128DA69009D5E0FF8C
:1076430090098AE0FEEEB5071F900987E0FF9009D5
:1076530051EFF0900988E0FF900952EFF09009890B
:10766300E0FF900953EFF0229009D6E0FF90098ADA
:10767300E0FEEEB5071F900987E0FF900954EFF095
:10768300900988E0FF900955EFF0900989E0FF9099
:107693000956EFF0229009D7E0FF90098AE0FEEE49
:1076A300B5071F900987E0FF900957EFF09009880D
:1076B300E0FF900958EFF0900989E0FF900959EF36
:1076C300F0229009D8E0FFEFB403057F5E128DA688
:1076D30022900770EBF0A3EAF0A3E9F0900770E0C3
:1076E300FBA3E0FAA3E0F912887690079EEFF090EF
:1076F3000770E0FBA3E0FAA3E0F9C003C002C001F6
:107703007B017A077977900650EBF0A3EAF0A3E9BF
:10771300F0D001D002D00312804E7B017A07797733
:10772300900798EBF0A3EAF0A3E9F0900773E0FB6E
:10773300A3E0FAA3E0F990079BEBF0A3EAF0A3E937
:10774300F0900776E4F0900776E0FFEFC3941050D3
:1077530030900798E0FBA3E475F0011250D3A9F031
:10776300FA124F73FF900773E0FBA3E475F0011265
:1077730050D3A9F0FAEF124FEC900776E004F080B3
:10778300C590079EE0FFEF24FBFF900776EFF09094
:10779300079EE0FF900776E0FEEEC39F503590070B
:1077A30070E0FBA3E0FAA3E0F9900776E0FF8F8295
:1077B300758300124F8CFF900773E0FBA3E475F011
:1077C300011250D3A9F0FAEF124FEC900776E004C0
:1077D300F080BC900773E0FBA3E0FAA3E0F9E412A6
:1077E3004FEC90079BE0FBA3E0FAA3E0F92290099A
:1077F300E7EBF0A3EAF0A3E9F09009EAEDF09009D2
:10780300EBE4F0A3E4F09009EBE0FEA3E0FFC3EFA9
:107813009405EE6480948040030278E89009EBE0DD
:10782300FEA3E0FF74582FF58274003EF583E0FF5A
:10783300EF60030278D79009EBE0FEA3E0FFEF7857
:1078430005C333CE33CED8F9FF745D2FF974003EF0
:10785300FA7B01C003C002C0019009E7E0FBA3E08B
:10786300FAA3E0F9900996EBF0A3EAF0A3E9F0900C
:1078730009EAE0FF7E00900999EEF0A3EFF0D00152
:10788300D002D003128B8A9009EBE0FEA3E0FFEF56
:10789300C43354E0245DF582E43400F583C083C02F
:1078A300829009EAE0FFD082D083E5822FF582E45B
:1078B3003583F583741AF09009EAE0FFEF04FF9033
:1078C30009EBE0FCA3E0FD74582DF58274003CF550
:1078D30083EFF0229009ECE004F070069009EBE0EE
:1078E30004F0027809224109D8004309D5000102B6
:1078F3004209D9070558082A0EFF00260DFF7570A7
:1079030012FF707C99FF7BA200FF0026000000009D
:10791300530000FFFE000E1197000000000000005E
:10792300000000000000602F00FEFFFE002A0000A0
:107933000000000000000000000000000000000044
:107943000000000000000000000000000000000034
:1079530000000000000000000049012DFFFE0004AC
:107963001100E00D1A490013FFFE000411958FCD9D
:107973001A5207CDFFFE000E109300000000000016
:107983000000000000004A09470001000A006403E8
:10799300E82710604007008000000000000000009E
:1079A30000000000000000000000000000000000D4
:1079B30000000000000000000000000000000000C4
:1079C30000000000000000000000000000000000B4
:1079D3000000000000000000900A14EBF0A3EAF09E
:1079E300A3E9F0900A14E0FBA3E0FAA3E0F9125331
:1079F3007600000000900A14E0FBA3E0FAA3E0F98C
:107A030075820475830012539000000000900A14DD
:107A1300E0FBA3E0FAA3E0F9758208758300125333
:107A23009067452301900A14E0FBA3E0FAA3E0F971
:107A330075820C758300125390EFCDAB89900A14B5
:107A4300E0FBA3E0FAA3E0F97582107583001253FB
:107A53009098BADCFE900A14E0FBA3E0FAA3E0F9E5
:107A630075821475830012539010325476900A175E
:107A7300E4F0A3E4F0900A17E0FEA3E0FFC3EF9461
:107A830040EE648094805035900A14E0FBA3E0FA42
:107A9300A3E0F9E92418F9EA3400FA900A17E0FEA2
:107AA300A3E0FFE92FF9EA3EFAE4124FEC900A183B
:107AB300E004F07006900A17E004F080B822900A00
:107AC3009FE4F0900393E0FFEFC3944040069003DC
:107AD30093743FF0C2AC900435E0FFEF7061900AFD
:107AE3009FE4F0900393E0FF900A9FE0FEEEC39FB4
:107AF300503290038FE0FBA3E0FAA3E0F9900A9FD2
:107B0300E0FF8F82758300124F8CFF900A9FE0FE87
:107B130074372EF582E43404F583EFF0900A9FE086
:107B230004F080BF900393E0FF900436EFF0C29916
:107B33009004357401F0900437E0FF8F99805D90D5
:107B43000A9FE4F0900393E0FF900A9FE0FEEEC3E8
:107B53009F504990038FE0FBA3E0FAA3E0F9900A5A
:107B63009FE0FF8F82758300124F8CFF900436E0F5
:107B7300FE74372EF582E43404F583EFF090043677
:107B8300E004F0900436E0FFEFC394404006900415
:107B930036743FF0900A9FE004F080A8D2AC2290A4
:107BA3000A0AEBF0A3EAF0A3E9F0900A0DEDF090D6
:107BB3000A0AE0FBA3E0FAA3E0F9124F73FF900A6D
:107BC3000EEFF0900A0DE4F0900A0AE0FBA3E0FA4E
:107BD300A3E0F9E4124FEC900A0EE0FFEF125469B0
:107BE3007BED027C560300007C7A7B017A007928C6
:107BF300C003C002C001900A0AE0FBA3E0FAA3E0BD
:107C0300F9E92408F9EA3400FA900996EBF0A3EABB
:107C1300F0A3E9F0900999E4F0A37414F0D001D033
:107C230002D003128B8A7B017A007928C003C00239
:107C3300C0017B017A00793D900773EBF0A3EAF072
:107C4300A3E9F0D001D002D0031276D490002474BB
:107C530001F0229009D8E0FFEFB404057F52128DA2
:107C6300A6900A0AE0FBA3E0FAA3E0F9E92409F9E4
:107C7300EA3400FA12852922900811E0FFEF64012B
:107C83006003027D44900811E4F08001227F017EAD
:107C9300007D007C00900816E0F8A3E0F9A3E0FA69
:107CA300A3E0FBC31252545003027D4490081AE030
:107CB300FCA3E0FDA3E0FEA3E0FF7B017A007900D3
:107CC3007800EF2BFFEE3AFEED39FDEC38FC90081F
:107CD3001A1253397B147A007900780090081AE05D
:107CE300FCA3E0FDA3E0FEA3E0FF12519FAC00ADB7
:107CF30001AE02AF037B007A0079007800C3125211
:107D030054703490081EE0FCA3E0FDA3E0FEA3E062
:107D1300FF7B017A0079007800EF2BFFEE3AFEED4E
:107D230039FDEC38FC90081E125339900822740177
:107D3300F09008287401F0900816125345000000D3
:107D43000022900A61EBF0A3EAF0A3E9F0900A6144
:107D5300E0FBA3E0FAA3E0F9124F73FFEFC4540F63
:107D6300FFEF540FFFEF1254697D76007DD00100C1
:107D7300007E0B900A61E0FBA3E0FAA3E0F9124F47
:107D830073FFEF540FFF9009D5EFF0900A61E0FB0A
:107D9300A3E0FAA3E0F9758201758300124F8CFF0B
:107DA300EFC4540FFFEF540FFF9009D6EFF0900A82
:107DB30061E0FBA3E0FAA3E0F97582017583001289
:107DC3004F8CFFEF540FFF9009D7EFF022900A6119
:107DD300E0FBA3E0FAA3E0F9124F73FFEF540FFFA8
:107DE3009009D9EFF0900A61E0FBA3E0FAA3E0F970
:107DF300758201758300124F8CFFEFC4540FFFEFA0
:107E0300540FFF9009DAEFF022900903EFF07BFFA4
:107E13007A8A79CFC003C002C0017B017A0979064F
:107E2300A801AC02AD03D001D002D0037E007F0ACB
:107E3300124F4D9009D5E0FFEF54FFFF90090CEF6F
:107E4300F09009D6E0FFEFC454F0FF9009D7E0FEAD
:107E5300EF4EFFEF54FFFF90090DEFF07B017A091E
:107E63007904C003C002C0017B017A09790A900832
:107E7300D7EBF0A3EAF0A3E9F09008DAE4F0A374F7
:107E830004F0D001D002D003127239900905E0FF4B
:107E930090090EEFF0900904E0FF90090FEFF090C6
:107EA3000903E0FFEF701290090A7410F07B017A66
:107EB3000979067D0A128C4B2290090A7411F07B12
:107EC300017A0979067D0A1277F12290095AEBF0BB
:107ED300A3EAF0A3E9F0900961E4F0A3E4F09009C8
:107EE30060E0FF14F0EF607E90095DE0FBA3E0FA31
:107EF300A3E0F9124F73FFEFC4540FFFEF540FFFCA
:107F0300128CE790095AE0FBA3E0FAA3E0F9900989
:107F130061E475F0011250D3ADF0FC8D828C83EFD8
:107F2300124FFE90095DE0FBA3E0FAA3E0F9124FC4
:107F330073FFEF540FFF128CE790095AE0FBA3E0A5
:107F4300FAA3E0F9900961E475F0011250D3ADF0A2
:107F5300FC8D828C83EF124FFE90095EE475F00175
:107F63001250BD027EE190095AE0FBA3E0FAA3E0C0
:107F7300F9900961E0FEA3E0FF8F828E83E4124F44
:107F8300FE90095AE0FBA3E0FAA3E0F9229009105E
:107F9300EFF07BFF7A8A79D9C003C002C0017B016D
:107FA3007A097913A801AC02AD03D001D002D00342
:107FB3007E007F0A124F4D9009D9E0FFEF4410FF76
:107FC300EF54FFFF900919EFF09009DAE0FFEFC4D7
:107FD30054F0FFEF54FFFF90091AEFF07B017A0989
:107FE3007911C003C002C0017B017A097917900897
:107FF300D7EBF0A3EAF0A3E9F09008DAE4F0A37476
:1080030004F0D001D002D003127239900912E0FFBC
:1080130090091BEFF0900911E0FF90091CEFF0901D
:108023000910E0FFEF70129009177410F07B017ACA
:108033000979137D0A128C4B229009177411F07B76
:10804300017A0979137D0A1277F12290064DEBF03C
:10805300A3EAF0A3E9F07B017A0679631279DB9056
:10806300064DE0FBA3E0FAA3E0F9128876EE339520
:10807300E0FDFC9008751253397B017A067963C0E1
:1080830003C002C00190064DE0FBA3E0FAA3E0F9B0
:10809300900872EBF0A3EAF0A3E9F0D001D002D08C
:1080A300031263BA7B017A067963C003C002C0017D
:1080B3007B017A067953900888EBF0A3EAF0A3E9F1
:1080C300F0D001D002D0031273E0900650E0FBA37E
:1080D300E0FAA3E0F9C003C002C0017B017A06798C
:1080E3005390095DEBF0A3EAF0A3E9F09009607403
:1080F30010F0D001D002D003127ECE900650E0FBE8
:10810300A3E0FAA3E0F922900A8DE4F0A3E4F0904F
:108113000A8DE0FEA3E0FFC3EF9403EE6480948036
:1081230040030281B3900A8DE0FEA3E0FF90095162
:1081330075F003EF1253B4EE75F003A42583F583B2
:10814300E4F0900A8DE0FEA3E0FF90095275F0037E
:10815300EF1253B4EE75F003A42583F583E4F09096
:108163000A8DE0FEA3E0FF90095375F003EF12536D
:10817300B4EE75F003A42583F583E4F0900A8DE053
:10818300FEA3E0FF90095275F003EF1253B4EE75AE
:10819300F003A42583F583E0FFEF4440FFEFF09065
:1081A3000A8EE004F07006900A8DE004F00281125A
:1081B30022C0E0C0F0C083C082C0D075D000C00030
:1081C300C001C002C003C004C005C006C00753AF4E
:1081D300FEE59A30E019539AFE900532E0FBA3E0E6
:1081E300FAA3E0F989828A83AF9B125493803BE51B
:1081F3009A30E136539AFD9007B6E0FF9007B7E057
:10820300FEEE6F601B9007B6E0FF74B82FF582E4B3
:108213003407F583E0FF8F9B9007B6E004F0800AF4
:108223009007B7E4F09007B6E4F043AF01D007D06E
:1082330006D005D004D003D002D001D000D0D0D0D6
:1082430082D083D0F0D0E032C0E0C0F0C083C082DF
:10825300C0D075D000C000C001C002C003C004C0BC
:1082630005C006C00753AFEFE58430E0195384FE21
:10827300900538E0FBA3E0FAA3E0F989828A83AF93
:1082830085125493803BE58430E1365384FD900599
:1082930086E0FF900587E0FEEE6F601B900586E0A9
:1082A300FF74882FF582E43405F583E0FF8F859012
:1082B3000586E004F0800A900587E4F0900586E4E3
:1082C300F043AF10D007D006D005D004D003D002BE
:1082D300D001D000D0D0D082D083D0F0D0E0329083
:1082E3000ABCEFF0900ABCE4F090047EE4F0900442
:1082F3007FE4F090047C74FFF090047D74FEF07BC7
:10830300017A047984900481EBF0A3EAF0A3E9F005
:108313007BFF7A8E79F790052FEBF0A3EAF0A3E9C0
:10832300F090049AE4F090049BE4F07BFF7A8E795A
:10833300DE900532EBF0A3EAF0A3E9F07B007A00CC
:108343007900900535EBF0A3EAF0A3E9F09004A4DB
:10835300E4F09004AAE4F09004A9E4F090052EE47C
:10836300F07BFF7A8F7910900538EBF0A3EAF0A346
:10837300E9F022787FE4F6D8FD75080075090075E9
:1083830081090283C30288DCE493A3F8E493A34046
:1083930003F68001F208DFF48029E493A3F854077D
:1083A300240CC8C333C4540F4420C8834004F45678
:1083B300800146F6DFE4800B0102040810204080B0
:1083C3009078E9E47E019360BCA3FF543F30E50954
:1083D300541FFEE493A360010ECF54C025E060A8B0
:1083E30040B8E493A3FAE493A3F8E493A3C8C58243
:1083F300C8CAC583CAF0A3C8C582C8CAC583CADFB1
:10840300E9DEE780BEC0E0C0F0C083C082C0D075A3
:10841300D000C000C001C002C003C004C005C00634
:10842300C00753AFF7E5AC30E01453ACFE900753ED
:10843300E5ADF07B017A077953128E1C803BE5ACE6
:1084430030E13653ACFD900761E0FF900762E0FE38
:10845300EE6F601B900761E0FF74632FF582E434D5
:1084630007F583E0FF8FAD900761E004F0800A9089
:108473000762E4F0900761E4F043AF08D007D00649
:10848300D005D004D003D002D001D000D0D0D08208
:10849300D083D0F0D0E032C0E0C0F0C083C082C04F
:1084A300D075D000C000C001C002C003C004C00525
:1084B300C006C007C2AC309818C29890052FE0FBE5
:1084C300A3E0FAA3E0F989828A83AF9912549380D7
:1084D30038309935C299900435E0FF900436E0FEB8
:1084E300EE6F601B900435E0FF74372FF582E434A0
:1084F30004F583E0FF8F99900435E004F0800A903F
:108503000436E4F0900435E4F0D2ACD007D006D0C2
:1085130005D004D003D002D001D000D0D0D082D077
:1085230083D0F0D0E032900A05EBF0A3EAF0A3E9A0
:10853300F0900A05E0FBA3E0FAA3E0F91287359077
:108543000A09EFF09009D8E0FFEFB40408900A0994
:10855300E0FF12899E900A09E0FFEF6409705490CE
:1085630000577401F0900A05E0FBA3E0FAA3E0F9D9
:10857300124F73FFEF642C6020900A05E0FBA3E029
:10858300FAA3E0F9124F73FFEF643A600C900A0606
:10859300E475F0011250BD80CC900A06E475F00139
:1085A3001250BD900A05E0FBA3E0FAA3E0F97D01B8
:1085B30012707C227B017A00791C12894090001D85
:1085C30074E0F07B017A01793612894090013774A7
:1085D300E0F0900025E4F0900026E4F0900053E4EE
:1085E300F0900054E4F0900027E4F0900057E4F09A
:1085F30090003CE4F0900052E4F0900A91E4F0A380
:10860300E4F0900A91E0FEA3E0FFC3EF9405EE646B
:108613008094805024900A91E0FEA3E0FF74582FC9
:10862300F58274003EF583E4F0900A92E004F07062
:1086330006900A91E004F080C922900A8BEFF09033
:108643000A8CEDF0900A8BE0FFEF12546986660006
:10865300867401868202869003869E0486AC05009A
:108663000086B9900A8CE0FFEF6003D29422C29493
:1086730022900A8CE0FFEF6003D2EB22C2EB229040
:108683000A8CE0FFEF6003D2EA22C2EA22900A8C4E
:10869300E0FFEF6003D2E922C2E922900A8CE0FFF7
:1086A300EF6003D29522C29522900A8CE0FFEF601F
:1086B30003D2C422C2C422900A31EFF0900A32EDF1
:1086C300F0900A33E4F0A3E4F0900A33E0FEA3E071
:1086D300FFC3EF9406EE648094805055900A33E014
:1086E300FEA3E0FF900A32E0FEEEA807088002C373
:1086F30013D8FCFFEF30E029900A33E0FEA3E0FF3C
:10870300900A33E0FCA3E0FDAE05900A31E0FDEDF5
:10871300A806088002C313D8FCFEEE5401FD12869E
:108723003D900A34E004F07006900A33E004F080D0
:108733009822900A41EBF0A3EAF0A3E9F0900A44EF
:10874300E4F0900A41E0FBA3E0FAA3E0F9124F73CF
:10875300FFEFC394304047900A41E0FBA3E0FAA344
:10876300E0F9124F73FFEFD394395032900A41E08E
:10877300FBA3E0FAA3E0F9124F73FFEF24D0FF90BD
:108783000A44E0FEEE75F00AA4FEEE2FFF900A44C1
:10879300EFF0900A42E475F0011250BD80A4900AF4
:1087A30044E0FF22C0E0C0F0C083C082C0D075D0D7
:1087B30000C000C001C002C003C004C005C006C0A1
:1087C30007C28D900816E0FCA3E0FDA3E0FEA3E042
:1087D300FF7B017A0079007800EF2BFFEE3AFEED84
:1087E30039FDEC38FC9008161253399008117401C6
:1087F300F0D007D006D005D004D003D002D001D0EA
:1088030000D0D0D082D083D0F0D0E0329009F3EE04
:10881300F0A3EFF09009F3E0FEA3E0FF9009F5EE7B
:10882300F0A3EFF09009F5E0FEA3E0FFD3EF94008F
:10883300EE9400403D9009F77401F0A3742CF0907E
:1088430009F7E0FEA3E0FFD3EF9400EE940040129B
:1088530000009009F8E024FFF09009F7E034FFF0FE
:1088630080DD9009F6E024FFF09009F5E034FFF095
:1088730080B2229009F9EBF0A3EAF0A3E9F09009A2
:10888300F9E0FBA3E0FAA3E0F99009FCEBF0A3EA1B
:10889300F0A3E9F09009FCE0FBA3E475F0011250AA
:1088A300D3A9F0FA124F73FFEF70E99009F9E0FBD7
:1088B300A3E0FAA3E0F9AE02AF019009FCE0FBA349
:1088C300E0FAA3E0F9AC02AD01C3ED9FFFEC9EFE1D
:1088D300EF24FFFFEE34FFFE221289F97FBC7E02F4
:1088E30012880F7BFF7A8D794B125B487FBC7E0227
:1088F30012880F7BFF7A8D795EC003C002C0017BB3
:10890300FF7A8D796C900141EBF0A3EAF0A3E9F0D3
:10891300D001D002D003125B487FBC7E0212880FC5
:10892300900828E0FFEFB40105900828E4F0127CDA
:108933007B7B017A047999128A5280E422900A6D32
:10894300EBF0A3EAF0A3E9F0900A6DE0FBA3E0FAF1
:10895300A3E0F97401124FEC900A6DE0FBA3E0FA77
:10896300A3E0F9758201758300E4124FFE900A6D4E
:10897300E0FBA3E0FAA3E0F9758202758300E41239
:108983004FFE900A6DE0FBA3E0FAA3E0F9758204C1
:108993007583001253900000000022900A9EEFF0AE
:1089A3009003937402F0900A9EE0FFEFC4540FFF0C
:1089B300EF25E02491F582E4348FF583E493FF906F
:1089C3000394EFF0900A9EE0FFEF540FFFEF25E0D2
:1089D3002491F582E4348FF583E493FF900395EFBC
:1089E300F07B017A03799490038FEBF0A3EAF0A371
:1089F300E9F0127AC122900A9BE4F0128AF3128FF3
:108A03006D128C137FBC7E0212880F7F00128E754D
:108A13007F02128F417F03128F577FBC7E02128821
:108A23000FD2AF7FBC7E0212880F7F001282E21248
:108A33008E90128EAA128EC4128AF3128D1B128F7D
:108A4300801285B712810A7FF47E0112880F22906B
:108A53000A29EBF0A3EAF0A3E9F0900A2CE4F090E2
:108A63000A29E0FBA3E0FAA3E0F97582027583000B
:108A7300124F8CFFEFB40127900A29E0FBA3E0FA21
:108A8300A3E0F9124F73FF128DA6900A29E0FBA30E
:108A9300E0FAA3E0F9758202758300E4124FFE2227
:108AA30056657273696F6E3A2025730D0A004D4146
:108AB30031305F76312E382E332E30002B43495020
:108AC3005243563A002B434349443A00FFFE000603
:108AD300009800000000FFFE000600980000000060
:108AE3000000000000000000000000000000000083
:108AF3007D007F0012863D7D007F0112863D7D0053
:108B03007F0212863D7D007F0312863D7D007F0438
:108B130012863D7D007F0512863D5391DF439220EF
:108B230053B3EF43B4105391EF43921053CBF74336
:108B3300CC0853CBFB43CC0453CBFD43CC02229054
:108B43000A35EBF0A3EAF0A3E9F0900A38EDF090D0
:108B53000A35E0FBA3E0FAA3E0F9124F73FFEFC479
:108B6300540FFFEF540FFFEF1254698B78008B8182
:108B73000100008B89900A38E0FF127E0C22900AD4
:108B830038E0FF127F9022900993EBF0A3EAF0A361
:108B9300E9F090099974FF75F0FF1250D3AFF0FE1E
:108BA300EF4E602A900996E0FBA3E475F0011250A2
:108BB300D3A9F0FA124F73FF900993E0FBA3E47576
:108BC300F0011250D3A9F0FAEF124FEC80C42290B7
:108BD3000A5EEBF0A3EAF0A3E9F0900A5EE0FBA3E0
:108BE300E0FAA3E0F9126E9E900A5EE0FBA3E0FABE
:108BF300A3E0F9124F73FF900A5EE0FBA3E0FAA330
:108C0300E0F9758201758300124F8CFD1286BA223A
:108C130090082412534500000000900828E4F090C7
:108C23000811E4F090081A12534500000000900860
:108C33001E12534500000000900822E4F09008162D
:108C43001253450000000022900A19EBF0A3EAF04A
:108C5300A3E9F0900A1CEDF0900A1CE0FF90039347
:108C6300EFF0900A19E0FBA3E0FAA3E0F990038F79
:108C7300EBF0A3EAF0A3E9F0127AC12243BA8090A1
:108C8300FFF2E4F090FFF07401F0A37423F090FF7F
:108C930004E4F090FF00E4F0A3E4F090FF02E4F0BA
:108CA300A37492F053BA7FC2A05395FE5396FE224B
:108CB300900A95EFF0900A95E0FFEFD394094010E6
:108CC300900A95E0FFEF2437FF900A96EFF0800EAD
:108CD300900A95E0FFEF2430FF900A96EFF0900A98
:108CE30096E0FF22900A99EFF0900A99E0FFEFD304
:108CF30094094010900A99E0FFEF2457FF900A9AD5
:108D0300EFF0800E900A99E0FFEF2430FF900A9A6B
:108D1300EFF0900A9AE0FF22C2A0C2A153B17F53A1
:108D2300B27F53B1BF53B2BF128C7F128D7A9008BA
:108D3300A8E4F09008A9E4F07B017A08799B1289F2
:108D43004090089C74E0F022496E697420636F6D53
:108D5300706C6574652E2E2E0D0A0056657273694C
:108D63006F6E3A2025730D0A004D4131305F763125
:108D73002E382E332E300043BA8090FFF2E4F09069
:108D8300FFF07401F0A37423F090FF14E4F090FF5C
:108D930010E4F0A3E4F090FF12E4F0A37492F05314
:108DA300BA7F22900A9DEFF09003937401F0900A2A
:108DB3009DE0FF900394EFF07B017A037994900395
:108DC3008FEBF0A3EAF0A3E9F0127AC122C0E0C06E
:108DD30083C082C0D075D000C007900A9CE0FFEF2B
:108DE3004440FF900A9CEFF0D007D0D0D082D083CC
:108DF300D0E032C0E0C083C082C0D075D000C007CD
:108E0300900A9CE0FFEF4480FF900A9CEFF0D007AC
:108E1300D0D0D082D083D0E032900A70EBF0A3EAB6
:108E2300F0A3E9F0900A70E0FBA3E0FAA3E0F97580
:108E330082027583007401124FFE22759A5075D712
:108E4300C075D6FD438E10538EF7438E04439202B2
:108E53005391FD43AF012275845075D3E875D2FF5A
:108E630043D12043D18043CA0853C9F743AF10D23B
:108E7300AF22900AB4EFF0900AB4E0FFEF7007530B
:108E8300A27F53A2BF2253A27F43A240227B017A37
:108E930003799490038FEBF0A3EAF0A3E9F0900435
:108EA30035E4F0128F29227B017A0779A59007A078
:108EB300EBF0A3EAF0A3E9F09007B6E4F0128E3EDC
:108EC300227B017A05794190053CEBF0A3EAF0A3FC
:108ED300E9F0900586E4F0128E5A22900AB9EFF079
:108EE300900AB9E0FF900499EFF07B017A04799935
:108EF300128E1C22900ABAEFF0900ABAE0FF900497
:108F03007AEFF07B017A04797812677322900ABBB7
:108F1300EFF0900ABBE0FF9004A3EFF07B017A042B
:108F230079A312558B22759850758920758BFD7521
:108F33008DFDD28E758E40C299C298D2AC22900A12
:108F4300B5EFF0900AB5E0FFEFB4020453BAFE2286
:108F530043BA0122900AB6EFF0900AB6E0FFEFB4ED
:108F6300030443BA042253BAFB22538E7F5389F07E
:108F7300758A00758C4CC28DD28CD2A9227B017A62
:108F83000779C51289409007C674E0F022003001CA
:108F930031023203330434053506360737083809FE
:0D8FA300390A410B420C430D440E450F46A8
:00000001FF
